:020000020000FC
:100000000C944C33189518951895189518951895C3
:100010001895189518951895189518951895189578
:100020001895189518951895189518951895189568
:100030001895189518951895189518951895189558
:100040001895189518951895189518951895189548
:100050000C94310D189518951895189518951895B4
:100060001895189518951895189518951895189528
:100070001895189518951895189518951895189518
:100080001895189518951895189518951895189508
:1000900018951895189518951895189518951895F8
:1000A00018951895189518951895189518951895E8
:1000B00018951895189518951895189518951895D8
:1000C00018951895189518951895189518951895C8
:1000D00018951895189518951895189518951895B8
:1000E00018951895189518951895189518951895A8
:1000F0001895189518951895189518951895189598
:100100001895189518951895189518951895189587
:100110001895189518951895189518950C94160D0E
:100120001895189518951895189518951895189567
:10013000189518950C948A0C18951895189518957B
:100140001895189518951895189518951895189547
:100150001895189518951895189518951895189537
:100160001895189518951895189518951895189527
:100170001895189518951895189518951895189517
:100180001895189518951895189518951895189507
:1001900018951895189518951895189518951895F7
:1001A00018951895189518951895189518951895E7
:1001B00018951895189518951895189518951895D7
:1001C00018951895189518951895189518951895C7
:1001D00018951895189518951895189518951895B7
:1001E00018951895189518951895189518951895A7
:1001F000189518951895189518951895D300053FDA
:10020000D30005BF000000000000803F561A20BD4B
:10021000000000009161F7BCBC5A4ABD6475A3BDE3
:10022000604FD6BD1B93A8BD3CCDD83CE3003F3EFC
:1002300011EA883EE3003F3E3CCDD83C1B93A8BD6D
:10024000604FD6BD6475A3BDBC5A4ABD9161F7BC71
:1002500014BEA1BD6FEDFCBDDC252FBEE9383F3FCC
:10026000DC252FBE6FEDFCBD14BEA1BD83E3D23EE5
:1002700083E3D2BE0000803FF671343E547AFFBB68
:10028000FF29ADBC2DEE49BD3C15D2BD94B644BE90
:10029000F6C03F3F94B644BE3C15D2BD2DEE49BDDD
:1002A000FF29ADBC547AFFBBE5FF3CBE6A8B31BE73
:1002B000D6704CBC0186593E0595A33E0186593E39
:1002C000D6704CBC6A8B31BEE5FF3CBE1F1F1F00C1
:1002D000000000001C1E1F1F1F1F1F1F1F1F1F1FAE
:1002E0001F1F1E1C00000000001F1F1F1F1F1F1FBD
:1002F0001F1F0F07070F1F1F1F1F1F1F00000000DA
:10030000001F1F1F1F1F1F00001F1F1F05000104CC
:1003100003022020052020FF000701040306000738
:10032000010603020506FF2020FF05070006030261
:100330000507000403020000012020FF0507010457
:100340000302050701030302050707042020050730
:100350000704030305070104202024212A2130215A
:1003600000003A27100074219523B823EF2343247B
:10037000A024DA2417255225AD25DF2518264A2684
:100380008426C026FE260000532F1000492C892CFD
:100390009E2CB32C222DF02D522EA02EB12EC22E2B
:1003A000D32EEB2E0A2F242F352F462F0000883214
:1003B0001000692FAE2FC32FD82F47301B317B3150
:1003C000D131E231F33104321C323F3259326A32D8
:1003D0007B32000113391039450339020339116D9D
:1003E000380B3238018B38010339010339010339E5
:1003F000028B38051F38016038016D38033B380225
:100400006D38036938FB03E333D000EE1EE22BD1D5
:1004100000EE1EE228D100EE1EE225D103E328D033
:1004200000EE1EE220D103E323D000EB14E01BD149
:1004300002E01ED000EB14E016D108E019D000EB6A
:1004400014E011D101E014D000EE1EE20CD100EE58
:100450001EE209D100EE1EE206D106E009D000EB53
:1004600014E001D10CE004D000EB14E0FCD00895BE
:100470008A93802FE4E4F6E000810F7B00830CE395
:1004800010E0F1D000916406007F00936406082F0D
:1004900002950F7010916406102B10936406E4E42B
:1004A000F6E00081006800830CE310E0DCD0E4E4B7
:1004B000F6E000810F7700830CE211E0D4D00091C8
:1004C0006406007F009364068F7000916406082B19
:1004D00000936406E4E4F6E00081006800830CE326
:1004E00010E0C1D0E4E4F6E000810F7700830CE275
:1004F00011E0B9D0899108958A93802FE4E4F6E061
:100500000081006400830CE310E0ADD0009164062C
:10051000007F00936406082F02950F701091640607
:10052000102B10936406E4E4F6E000810068008379
:100530000CE310E098D0E4E4F6E000810F7700834C
:100540000CE211E090D000916406007F00936406F5
:100550008F7000916406082B00936406E4E4F6E0D3
:100560000081006800830CE310E07DD0E4E4F6E055
:1005700000810F7700830CE211E075D08991089516
:100580000E94CB36C801A0E007C0B0E0FC01EA0F32
:10059000FB1F0081B1DFA395B0E0FC01EA0FFB1F58
:1005A0000081002311F0A13180F3E4E00C94DC36EB
:1005B0005FDF01E215E2E4DF08950BEC00935200E7
:1005C00008E000935000E1E5F0E0008103FFFBCF7D
:1005D00003EC00935500E0E5F0E00081006100834A
:1005E000E1E5F0E0008104FFFBCF08ED04BF04E08B
:1005F00000934000E0E5F0E000810E7F0083089565
:1006000000E00093010202E20093020203E0009383
:10061000040201E00093200200E200932102E0E0E6
:10062000F2E0008101600083089501E00093280258
:1006300000E300932902089501E00093300208E3EB
:100640000093310208950DE00093200300E400932D
:10065000210300E00093220300E50093240300E758
:100660000093280308950150104098018901232B1D
:10067000D1F708958A93802F04C008EE1DEF0E94E1
:100680003B158A95082F802F0023B9F7899108958B
:100690000E94C73682E035C0482F50E0440F551FF6
:1006A000440F551FFA01E75CFA4D0080118022804B
:1006B0003380482F50E0440F551F440F551FFA0157
:1006C000E35CFA4D0082118222823382482F50E08F
:1006D000440F551F440F551FFA01E35DFA4D00808A
:1006E000118022803380482F50E0440F551F440F63
:1006F000551FFA01EF5CFA4D00821182228233828B
:100700008A95813048F6EDE3F5E200831183228378
:100710003383EDE3F5E24081518162817381ECEF37
:10072000F1E005911591259134910E944F35E1E357
:10073000F5E2008311832283338381E04FC0082FC9
:1007400010E0000F111F000F111FF801E450FE4FC1
:100750004591559165917491082F10E0000F111F7C
:10076000000F111FF801E35CFA4D00811181228115
:1007700033810E944F3528013901082F10E0000F06
:10078000111F000F111FF801E85FFD4F45915591B2
:1007900065917491082F10E0000F111F000F111FB9
:1007A000F801EF5CFA4D00811181228133810E94B2
:1007B0004F35A801B901820193010E943235E1E36E
:1007C000F5E240815181628173810E94EE34E1E360
:1007D000F5E200831183228333838395833008F409
:1007E000AECFE1E3F5E20081118122813381E8E0BF
:1007F0000C94D8360E94C73682E035C0482F50E0AE
:10080000440F551F440F551FFA01EF5AFA4D00804F
:10081000118022803380482F50E0440F551F440F31
:10082000551FFA01EB5AFA4D00821182228233825F
:10083000482F50E0440F551F440F551FFA01EB5B42
:10084000FA4D0080118022803380482F50E0440F01
:10085000551F440F551FFA01E75BFA4D00821182C4
:10086000228233828A95813048F6E5E5F5E20083FD
:10087000118322833383E5E5F5E240815181628172
:100880007381ECEFF1E005911591259134910E946F
:100890004F35E9E4F5E2008311832283338381E05D
:1008A0004FC0082F10E0000F111F000F111FF8019B
:1008B000E450FE4F4591559165917491082F10E0D9
:1008C000000F111F000F111FF801EB5AFA4D0081A4
:1008D0001181228133810E944F3528013901082F6F
:1008E00010E0000F111F000F111FF801E85FFD4F0E
:1008F0004591559165917491082F10E0000F111FDB
:10090000000F111FF801E75BFA4D00811181228170
:1009100033810E944F35A801B901820193010E94E1
:100920003235E9E4F5E240815181628173810E94B0
:10093000EE34E9E4F5E20083118322833383839567
:10094000833008F4AECFE9E4F5E200811181228121
:100950003381E8E00C94D8360E94C73682E035C077
:10096000482F50E0440F551F440F551FFA01E75917
:10097000FA4D0080118022803380482F50E0440FD0
:10098000551F440F551FFA01E359FA4D0082118299
:1009900022823382482F50E0440F551F440F551FC9
:1009A000FA01E35AFA4D0080118022803380482FEB
:1009B00050E0440F551F440F551FFA01EF59FA4DEF
:1009C00000821182228233828A95813048F6EDE6D8
:1009D000F5E20083118322833383EDE6F5E2408163
:1009E000518162817381ECEFF1E0059115912591C0
:1009F00034910E944F35E1E6F5E2008311832283B2
:100A0000338381E04FC0082F10E0000F111F000F4B
:100A1000111FF801E450FE4F459155916591749175
:100A2000082F10E0000F111F000F111FF801E359EC
:100A3000FA4D00811181228133810E944F352801B6
:100A40003901082F10E0000F111F000F111FF801CE
:100A5000E85FFD4F4591559165917491082F10E025
:100A6000000F111F000F111FF801EF59FA4D0081FF
:100A70001181228133810E944F35A801B901820181
:100A800093010E943235E1E6F5E2408151816281B5
:100A900073810E94EE34E1E6F5E200831183228344
:100AA00033838395833008F4AECFE1E6F5E200812D
:100AB000118122813381E8E00C94D8360E94CA3635
:100AC00080E090E0A0E0B0E04EE0442E1BC0442D5A
:100AD00050E0440F551F440F551FFA01EB58FA4DD3
:100AE0000080118022803380442D50E0440F551F38
:100AF000440F551FFA01E758FA4D008211822282F5
:100B000033824A9441E0441610F7E9E7F5E20083A6
:100B1000118322833383442423C0042D10E0000F6B
:100B2000111F000F111FF801EC5EFD4F459155910B
:100B300065917491042D10E0000F111F000F111F1B
:100B4000F801E758FA4D00811181228133810E941A
:100B50004F35AC01BD010E94EE34C801D901439468
:100B60000FE04016D0F28C019D01E5E00C94DB36DD
:100B70000E94CA3680E090E0A0E0B0E04EE0442E53
:100B80001BC0442D50E0440F551F440F551FFA0160
:100B9000EF54FA4D0080118022803380442D50E0C4
:100BA000440F551F440F551FFA01EB54FA4D0082B4
:100BB0001182228233824A9441E0441610F7E5EB19
:100BC000F5E20083118322833383442423C0042D60
:100BD00010E0000F111F000F111FF801EC5EFD4F18
:100BE0004591559165917491042D10E0000F111FEE
:100BF000000F111FF801EB54FA4D00811181228181
:100C000033810E944F35AC01BD010E94EE34C80112
:100C1000D90143940FE04016D0F28C019D01E5E02C
:100C20000C94DB360E94CA3680E090E0A0E0B0E091
:100C30004EE0442E1BC0442D50E0440F551F440F7E
:100C4000551FFA01E351FA4D008011802280338054
:100C5000442D50E0440F551F440F551FFA01EF502B
:100C6000FA4D00821182228233824A9441E0441676
:100C700010F7E1EFF5E200831183228333834424EC
:100C800023C0042D10E0000F111F000F111FF801E9
:100C9000EC5EFD4F4591559165917491042D10E0E6
:100CA000000F111F000F111FF801EF50FA4D0081C6
:100CB0001181228133810E944F35AC01BD010E9418
:100CC000EE34C801D90143940FE04016D0F28C01F4
:100CD0009D01E5E00C94DB360E94CA3680E090E08E
:100CE000A0E0B0E046E0442E1BC0442D50E0440F8D
:100CF000551F440F551FFA01E75DF94D0080118023
:100D000022803380442D50E0440F551F440F551F5F
:100D1000FA01E35DF94D00821182228233824A9406
:100D200041E0441610F7EDE2F6E2008311832283DE
:100D30003383442423C0042D10E0000F111F000F43
:100D4000111FF801E05BFD4F45915591659174913C
:100D5000042D10E0000F111F000F111FF801E35DBB
:100D6000F94D00811181228133810E944F35AC0100
:100D7000BD010E94EE34C801D901439407E040163A
:100D8000D0F28C019D01E5E00C94DB360E94CA365E
:100D900080E090E0A0E0B0E046E0442E1BC0442D8F
:100DA00050E0440F551F440F551FFA01EB5BF94DFE
:100DB0000080118022803380442D50E0440F551F65
:100DC000440F551FFA01E75BF94D00821182228220
:100DD00033824A9441E0441610F7E9E4F6E20083D6
:100DE000118322833383442423C0042D10E0000F99
:100DF000111F000F111FF801E05BFD4F4591559148
:100E000065917491042D10E0000F111F000F111F48
:100E1000F801E75BF94D00811181228133810E9445
:100E20004F35AC01BD010E94EE34C801D901439495
:100E300007E04016D0F28C019D01E5E00C94DB3612
:100E40000E94CA3680E090E0A0E0B0E046E0442E88
:100E50001BC0442D50E0440F551F440F551FFA018D
:100E6000EF59F94D0080118022803380442D50E0ED
:100E7000440F551F440F551FFA01EB59F94D0082DD
:100E80001182228233824A9441E0441610F7E5E64B
:100E9000F6E20083118322833383442423C0042D8C
:100EA00010E0000F111F000F111FF801E05BFD4F54
:100EB0004591559165917491042D10E0000F111F1B
:100EC000000F111FF801EB59F94D008111812281AA
:100ED00033810E944F35AC01BD010E94EE34C80140
:100EE000D901439407E04016D0F28C019D01E5E062
:100EF0000C94DB360E94C736842FA52F0E948F34B6
:100F0000482F50E0440F551F440F551FFA01EF576B
:100F1000F94D40815181628173810E9432352801EF
:100F200039010A2F10E020E030E00E949A34A80135
:100F3000B901820193010E94C835482F50E0440F47
:100F4000551F440F551FFA01EF57F94D408151814C
:100F5000628173810E94EE3490E0880F991F880FA0
:100F6000991FFC01EF57F94D0083118322833383CE
:100F7000E8E00C94D8360E94C73681E035C0482F8F
:100F800050E0440F551F440F551FFA01EB53F94D24
:100F90000080118022803380482F50E0440F551F7D
:100FA000440F551FFA01E753F94D00821182228246
:100FB0003382482F50E0440F551F440F551FFA014C
:100FC000E354F94D0080118022803380482F50E097
:100FD000440F551F440F551FFA01EF53F94D00827E
:100FE0001182228233828A95813048F6E9ECF6E25A
:100FF0000083118322833383E9ECF6E2408151813F
:1010000062817381ECE6F2E00591159125913491AE
:101010000E944F35E1ECF6E2008311832283338393
:1010200081E04FC0082F10E0000F111F000F111FAB
:10103000F801E459FD4F4591559165917491082F40
:1010400010E0000F111F000F111FF801E753F94DB9
:1010500000811181228133810E944F35280139019D
:10106000082F10E0000F111F000F111FF801EC589E
:10107000FD4F4591559165917491082F10E0000F37
:10108000111F000F111FF801EF53F94D008111815D
:10109000228133810E944F35A801B9018201930159
:1010A0000E943235E1ECF6E2408151816281738128
:1010B0000E94EE34E1ECF6E2008311832283338355
:1010C0008395823008F4AECFE1ECF6E20081118125
:1010D00022813381E8E00C94D8360E94C73681E043
:1010E00035C0482F50E0440F551F440F551FFA01DB
:1010F000EB52F94D0080118022803380482F50E060
:10110000440F551F440F551FFA01E752F94D008255
:10111000118222823382482F50E0440F551F440F22
:10112000551FFA01E353F94D00801180228033806E
:10113000482F50E0440F551F440F551FFA01EF523E
:10114000F94D00821182228233828A95813048F6DD
:10115000E9EDF6E20083118322833383E9EDF6E2C1
:101160004081518162817381ECE6F2E00591159135
:10117000259134910E944F35E1EDF6E20083118311
:101180002283338381E04FC0082F10E0000F111F2E
:10119000000F111FF801E459FD4F459155916591DC
:1011A0007491082F10E0000F111F000F111FF8019C
:1011B000E752F94D00811181228133810E944F3520
:1011C00028013901082F10E0000F111F000F111F17
:1011D000F801EC58FD4F4591559165917491082F98
:1011E00010E0000F111F000F111FF801EF52F94D11
:1011F00000811181228133810E944F35A801B901FC
:10120000820193010E943235E1EDF6E24081518185
:10121000628173810E94EE34E1EDF6E20083118376
:10122000228333838395823008F4AECFE1EDF6E27A
:101230000081118122813381E8E00C94D8360E942C
:10124000C73681E035C0482F50E0440F551F440F8A
:10125000551FFA01EB51F94D008011802280338037
:10126000482F50E0440F551F440F551FFA01E75116
:10127000F94D0082118222823382482F50E0440FC0
:10128000551F440F551FFA01E352F94D008011809C
:1012900022803380482F50E0440F551F440F551FC4
:1012A000FA01EF51F94D00821182228233828A9530
:1012B000813048F6E9EEF6E200831183228333831E
:1012C000E9EEF6E24081518162817381ECE6F2E061
:1012D00005911591259134910E944F35E1EEF6E28A
:1012E000008311832283338381E04FC0082F10E0F5
:1012F000000F111F000F111FF801E459FD4F459118
:10130000559165917491082F10E0000F111F000F87
:10131000111FF801E751F94D0081118122813381BC
:101320000E944F3528013901082F10E0000F111FCE
:10133000000F111FF801EC58FD4F45915591659133
:101340007491082F10E0000F111F000F111FF801FA
:10135000EF51F94D00811181228133810E944F3577
:10136000A801B901820193010E943235E1EEF6E253
:1013700040815181628173810E94EE34E1EEF6E298
:1013800000831183228333838395823008F4AECFA8
:10139000E1EEF6E20081118122813381E8E00C94D4
:1013A000D8360E94CA3680E090E0A0E0B0E04AE083
:1013B000442E1BC0442D50E0440F551F440F551FB1
:1013C000FA01E351F94D0080118022803380442DD1
:1013D00050E0440F551F440F551FFA01EF50F94DCF
:1013E00000821182228233824A9441E0441610F72F
:1013F000E1EFF6E20083118322833383442423C088
:10140000042D10E0000F111F000F111FF801E45808
:10141000FD4F4591559165917491042D10E0000F99
:10142000111F000F111FF801EF50F94D00811181BC
:10143000228133810E944F35AC01BD010E94EE3400
:10144000C801D90143940BE04016D0F28C019D01F4
:10145000E5E00C94DB360E94CA3680E090E0A0E024
:10146000B0E04AE0442E1BC0442D50E0440F551F0D
:10147000440F551FFA01E75EF84D0080118022806D
:101480003380442D50E0440F551F440F551FFA017F
:10149000E35EF84D00821182228233824A9441E059
:1014A000441610F7EDE1F7E20083118322833383C2
:1014B000442423C0042D10E0000F111F000F111F42
:1014C000F801E458FD4F4591559165917491042DB3
:1014D00010E0000F111F000F111FF801E35EF84D1F
:1014E00000811181228133810E944F35AC01BD0101
:1014F0000E94EE34C801D90143940BE04016D0F2AB
:101500008C019D01E5E00C94DB360E94CA3680E038
:1015100090E0A0E0B0E04AE0442E1BC0442D50E033
:10152000440F551F440F551FFA01EB5BF84D008027
:10153000118022803380442D50E0440F551F440F0A
:10154000551FFA01E75BF84D008211822282338237
:101550004A9441E0441610F7E9E4F7E2008311836E
:1015600022833383442423C0042D10E0000F111F75
:10157000000F111FF801E458FD4F459155916591F9
:101580007491042D10E0000F111F000F111FF801BE
:10159000E75BF84D00811181228133810E944F3534
:1015A000AC01BD010E94EE34C801D90143940BE0A7
:1015B0004016D0F28C019D01E5E00C94DB360E94D0
:1015C000CA3680E090E0A0E0B0E048E0442E1BC0C6
:1015D000442D50E0440F551F440F551FFA01EF589A
:1015E000F84D0080118022803380442D50E0440F5C
:1015F000551F440F551FFA01EB58F84D0082118218
:10160000228233824A9441E0441610F7E5E7F7E27C
:101610000083118322833383442423C0042D10E0EC
:10162000000F111F000F111FF801E855FD4F4591E4
:10163000559165917491042D10E0000F111F000F5A
:10164000111FF801EB58F84D00811181228133817F
:101650000E944F35AC01BD010E94EE34C801D90192
:10166000439409E04016D0F28C019D01E5E00C9412
:10167000DB360E94CA3680E090E0A0E0B0E048E0AF
:10168000442E1BC0442D50E0440F551F440F551FDE
:10169000FA01EB56F84D0080118022803380442DF2
:1016A00050E0440F551F440F551FFA01E756F84DFF
:1016B00000821182228233824A9441E0441610F75C
:1016C000E9E9F7E20083118322833383442423C0B2
:1016D000042D10E0000F111F000F111FF801E85535
:1016E000FD4F4591559165917491042D10E0000FC7
:1016F000111F000F111FF801E756F84D00811181ED
:10170000228133810E944F35AC01BD010E94EE342D
:10171000C801D901439409E04016D0F28C019D0123
:10172000E5E00C94DB360E94CA3680E090E0A0E051
:10173000B0E048E0442E1BC0442D50E0440F551F3C
:10174000440F551FFA01E754F84D008011802280A4
:101750003380442D50E0440F551F440F551FFA01AC
:10176000E354F84D00821182228233824A9441E090
:10177000441610F7EDEBF7E20083118322833383E5
:10178000442423C0042D10E0000F111F000F111F6F
:10179000F801E855FD4F4591559165917491042DDF
:1017A00010E0000F111F000F111FF801E354F84D56
:1017B00000811181228133810E944F35AC01BD012E
:1017C0000E94EE34C801D901439409E04016D0F2DA
:1017D0008C019D01E5E00C94DB361091480001E09E
:1017E000009348002091A0003091A2000091A20037
:1017F0000C7F04600093A2004FB77894E8E4F0E017
:101800000081016000835091CD01EF93FF930F930E
:101810002F93EBECF1E008ED21E004BF20832F9142
:101820000F91FF91EF9103E00093CD018895109304
:1018300048002093A0003093A2005093CD014FBFE9
:101840000895EFECF1E0008107FDFBCF0895F9DF8B
:10185000EFECF1E0008101FF11C006E30093CA0143
:10186000EF93FF930F932F93EBECF1E008ED21E062
:1018700004BF20832F910F91FF91EF9108959A93C8
:101880008A93C801DEDF082F0093C001892F8F7172
:101890008093C10100E00093C20106E00093CA01F9
:1018A000EF93FF930F932F93EBECF1E008ED21E022
:1018B00004BF20832F910F91FF91EF910091C401FC
:1018C0008991999108950E94CC36C801A22F00E019
:1018D0000093060900E000934608B9DF03E3009394
:1018E000CA01082F0093C001892F8F718093C10115
:1018F00000E00093C201A093C40105E30093CA0174
:101900006CDF03E00093060901E000934608E3E082
:101910000C94DD369A938A93FA93EA930A927A9317
:101920006A935A934A933A932A931A930A930FB657
:10193000E0E0F2E00081046000830091FA29039561
:101940000093FA29083018F000E00093FA2900917A
:10195000FD290023B1F10091412910914229212F45
:10196000220F220B322F4091FA2950E0440F551FCD
:10197000440F551FFA01EF51F74D408151816281AB
:101980007381400F511F621F731F40835183628315
:1019900073838091572990915829019680935729F4
:1019A000909358290091512910915229801791073D
:1019B00041F400E00093FD2910E0009357291093B3
:1019C0005829E5E2F3E0008100FF0EC00091FA29FA
:1019D00010E0000F111FF801EF51F84D0081118147
:1019E0000093380310933903E5E2F3E0008101FF2F
:1019F0000EC00091FA2910E0000F111FF801EF5FEF
:101A0000F74D0081118100933A0310933B030FBE01
:101A10000991199129913991499159916991799136
:101A20000990E991F9918991999118954A933A937E
:101A30002A931A930A934FB7009110021091110242
:101A400020911D2A30911E2A021B130B009341295D
:101A5000109342294FBF09911991299139914991C8
:101A600018957A926A925A924A929A938A93FA9322
:101A7000EA933A922A921A920A927A936A935A9322
:101A80004A933A932A931A930A939FB70091FD2998
:101A9000002309F07FC40091182A0E5F0093152AD5
:101AA00080E034C05091152A482F642F082F10E091
:101AB000000F111F000F111FF801EF51F74D0081AA
:101AC0001181228133814091F5290E940234462FF1
:101AD00011DA0E949C34282F30E0220F331FF901C5
:101AE000EF5DF64D0083118300E010E020E030E070
:101AF000482F50E0440F551F440F551FFA01EF5176
:101B0000F74D00831183228333838395883050F20D
:101B10000FEF0093FD2900E010E020E030E0E1E667
:101B2000F9E20083118322833383EDE5F9E2008338
:101B3000118322833383E9E5F9E200831183228351
:101B4000338300E010E020E030E0EFE1FAE20083D0
:101B500011832283338380E0CFC0082F10E0000F71
:101B6000111FF801EF5DF64D00811181212F220F29
:101B7000220B322F0E948F3428013901082F10E0E8
:101B8000000F111FF801EF5DF64D00811181212F2B
:101B9000220F220B322F0E948F34A201B3010E9428
:101BA0004F35EFE1FAE240815181628173810E94F9
:101BB000EE34EFE1FAE20083118322833383E9E517
:101BC000F9E200811181228133810E948F34280142
:101BD0003901082F10E0000F111FF801EF5DF64DDD
:101BE00000811181212F220F220B322F0E948F346E
:101BF000482F50E0440F551F440F551FFA01EF5D69
:101C0000F74D40815181628173810E944F35A2015D
:101C1000B3010E94EE340E949C34E9E5F9E20083AE
:101C2000118322833383EDE5F9E200811181228162
:101C300033810E948F3428013901082F10E0000FF2
:101C4000111FF801EF5DF64D00811181212F220F48
:101C5000220B322F0E948F34482F50E0440F551F23
:101C6000440F551FFA01EF59F74D408151816281B0
:101C700073810E944F35A201B3010E94EE340E948D
:101C80009C34EDE5F9E20083118322833383E1E69E
:101C9000F9E200811181228133810E948F34280171
:101CA0003901082F10E0000F111FF801EF5DF64D0C
:101CB00000811181212F220F220B322F0E948F349D
:101CC000482F50E0440F551F440F551FFA01EF55A0
:101CD000F74D40815181628173810E944F35A2018D
:101CE000B3010E94EE340E949C34E1E6F9E20083E5
:101CF0001183228333838395883008F42ECF40E00C
:101D000050E060E071E4EFE1FAE2008111812281AC
:101D100033810E94C8350E94333BEFE1FAE2008331
:101D20001183228333830091F929013099F4EFE183
:101D3000FAE200811181228133810E949C3440911A
:101D40005329509154290E94AE3300931B2A1093BB
:101D50001C2A14C0EFE1FAE2008111812281338153
:101D60000E949C344091532950915429440F551F8F
:101D70000E94AE3300931B2A10931C2AE9E5F9E276
:101D80000081118122813381EDE6F9E20083118324
:101D900022833383EDE5F9E20081118122813381D1
:101DA000E1E7F9E20083118322833383E1E6F9E27C
:101DB0000081118122813381E9E7F9E200831183F7
:101DC000228333830091FC29002339F100E0009342
:101DD000FC29EDE6F9E20081118122813381E1E8FD
:101DE000F9E20083118322833383E1E7F9E2008182
:101DF000118122813381EDE7F9E20083118322838F
:101E00003383E9E7F9E20081118122813381E5E83A
:101E1000F9E20083118322833383E1E8F9E2008150
:101E2000118122813381EDE6F9E2408151816281A5
:101E30007381401B510B620B730B40835183628390
:101E40007383EDE7F9E20081118122813381E1E7BB
:101E5000F9E24081518162817381401B510B620B19
:101E6000730B4083518362837383E5E8F9E2008159
:101E7000118122813381E9E7F9E240815181628158
:101E80007381401B510B620B730B40835183628340
:101E900073830091042A002309F05DC10091F929A0
:101EA000033009F458C10091F929013009F0ADC09F
:101EB0000091132A0130B9F5EDE6F9E200811181B4
:101EC000228133810E948F340E9448030E949C34F7
:101ED000EDE9F9E20083118322833383E1E7F9E23C
:101EE00000811181228133810E948F340E94FA0384
:101EF0000E949C34E1EAF9E2008311832283338358
:101F0000E9E7F9E200811181228133810E948F3457
:101F10000E94AC040E949C34E9E9F9E20083118339
:101F2000228333833CC10091132A0230B9F5EDE6D8
:101F3000F9E200811181228133810E948F340E9455
:101F40005E050E949C34EDE9F9E20083118322834F
:101F50003383E1E7F9E200811181228133810E941C
:101F60008F340E94B8050E949C34E1EAF9E20083B4
:101F7000118322833383E9E7F9E200811181228111
:101F800033810E948F340E9412060E949C34E9E93A
:101F9000F9E2008311832283338301C1EDE6F9E284
:101FA00000811181228133810E948F340E946C064E
:101FB0000E949C34EDE9F9E200831183228333838C
:101FC000E1E7F9E200811181228133810E948F349F
:101FD0000E94C6060E949C34E1EAF9E20083118364
:101FE00022833383E9E7F9E2008111812281338181
:101FF0000E948F340E9420070E949C34E9E9F9E294
:102000000083118322833383CAC00091132A0130D5
:10201000B1F5EDE6F9E200811181228133810E9460
:102020008F340E94BB070E949C34EDE9F9E20083E3
:10203000118322833383E1E7F9E200811181228158
:1020400033810E948F340E946D080E949C34E1EA23
:10205000F9E20083118322833383E9E7F9E2008107
:102060001181228133810E948F34E9D80E949C34EF
:10207000E9E9F9E2008311832283338390C0009160
:10208000132A0230A1F5EDE6F9E2008111812281E7
:1020900033810E948F3493DA0E949C34EDE9F9E297
:1020A0000083118322833383E1E7F9E20081118108
:1020B000228133810E948F34DCDA0E949C34E1EA71
:1020C000F9E20083118322833383E9E7F9E2008197
:1020D0001181228133810E948F3425DB0E949C3440
:1020E000E9E9F9E2008311832283338358C0EDE6E6
:1020F000F9E200811181228133810E948F3451D90C
:102100000E949C34EDE9F9E200831183228333833A
:10211000E1E7F9E200811181228133810E948F344D
:102120009AD90E949C34E1EAF9E200831183228368
:102130003383E9E7F9E200811181228133810E9432
:102140008F34E3D90E949C34E9E9F9E200831183DA
:102150002283338324C0EDE6F9E2008111812281DC
:102160003381EDE9F9E20083118322833383E1E7D0
:10217000F9E20081118122813381E1EAF9E20083F1
:10218000118322833383E9E7F9E2008111812281FF
:102190003381E9E9F9E200831183228333830091DB
:1021A0000E2A009500930E2A00910E2A002309F0B2
:1021B000CDC0EDE9F9E20081118122813381E9EAA4
:1021C000F9E24081518162817381040F151F261F3E
:1021D000371FE5EBF9E20083118322833383E1EAC1
:1021E000F9E20081118122813381EDEAF9E2408137
:1021F000518162817381040F151F261F371FE9EB80
:10220000F9E20083118322833383E9E9F9E2008153
:10221000118122813381E5EAF9E2408151816281B5
:102220007381040F151F261F371FE1EBF9E20083AE
:1022300011832283338300910F2A009500930F2A84
:1022400000910F2A002309F05CC084E00091162A57
:10225000801BE5EBF9E20081118122813381EDEBF6
:10226000F9E24081518162817381040F151F261F9D
:10227000371F482F50E060E070E00E942D34E5E603
:10228000F9E20083118322833383E9EBF9E20081D1
:10229000118122813381E1ECF9E240815181628137
:1022A0007381040F151F261F371F482F50E060E071
:1022B00070E00E942D34E9E6F9E200831183228365
:1022C0003383E1EBF9E20081118122813381E5EC76
:1022D000F9E24081518162817381040F151F261F2D
:1022E000371F482F50E060E070E00E942D34E5E792
:1022F000F9E200831183228333830FEF0093102AC6
:1023000049C0E5EBF9E20081118122813381EDEBD7
:10231000F9E20083118322833383E9EBF9E2008140
:10232000118122813381E1ECF9E200831183228360
:102330003383E1EBF9E20081118122813381E5EC05
:10234000F9E2008311832283338324C0EDE9F9E2AB
:102350000081118122813381E9EAF9E2008311834E
:1023600022833383E1EAF9E2008111812281338102
:10237000EDEAF9E20083118322833383E9E9F9E28C
:102380000081118122813381E5EAF9E20083118322
:10239000228333839FBF09911991299139914991E2
:1023A0005991699179910990199029903990E99101
:1023B000F9918991999149905990699079901895DE
:1023C0000E94CB3600E40E943802AFEF80E002C0EA
:1023D000A69583958830A8F4BA2F90E005C000E058
:1023E0000E947C02B6959395983090F7BB2311F02C
:1023F00001E001C000E0002391F70FE10E947C02A0
:10240000F1CFE4E00C94DC369A938A9300E40E94C6
:10241000380280E008C090E0FC01E453FD4F0491D5
:102420000E947C0283958034B0F38991999108953C
:102430000E94CB36D80180E090E02FC00DE210E082
:10244000AC010E949A330A0F1B1F212F220F220B6F
:10245000322F0E948F3440E050E064EB73E40E941E
:10246000693630F440E050E064EB73EC0E94EE34E7
:1024700045E35AEF6EE87CE30E944F350E944833F3
:10248000AC01440F551F440F551FFA01EF55F74D8E
:1024900000831183228333830196883000E0900704
:1024A0006CF2E4E00C94DC360E94CB36D80180E07C
:1024B00090E02FC00DE210E0AC010E949A330A0FA9
:1024C0001B1F212F220F220B322F0E948F3440E03E
:1024D00050E064EB73E40E94693630F440E050E071
:1024E00064EB73EC0E94EE3445E35AEF6EE87CE354
:1024F0000E944F350E94653AAC01440F551F440FAE
:10250000551FFA01EF5DF74D00831183228333835A
:102510000196883000E090076CF2E4E00C94DC3621
:102520000E94CB36D80180E090E02FC00DE210E091
:10253000AC010E949A330A0F1B1F212F220F220B7E
:10254000322F0E948F3440E050E064EB73E40E942D
:10255000693630F440E050E064EB73EC0E94EE34F6
:1025600045E35AEF6EE87CE30E944F350E94483302
:10257000AC01440F551F440F551FFA01EF59F74D99
:1025800000831183228333830196883000E0900713
:102590006CF2E4E00C94DC360E94C336D8010BEDFB
:1025A000802E0FE0902E09E4A02E0FE3B02E80E0E5
:1025B00090E048C08D01212F220F220B322F0E9464
:1025C0008F34280139018C01212F220F220B322F49
:1025D0000E948F34A401B5010E944F350E94653AD4
:1025E000A201B3010E944F35280139018D01212F2D
:1025F000220F220B322F0E948F34A201B3010E94BE
:10260000EE342801390108EF17E00A1B1B0B980173
:1026100044E050E089010E94C633212F220F220B93
:10262000322F0E948F34A201B3010E94EE340E9427
:102630009C349C01220F331FF901EF5FF74D00839B
:1026400011830196883000E090070CF4B3CFECE0E2
:102650000C94D4360E94C5364801D90180E090E040
:1026600046C00DE210E0AC010E949A33A801480D6B
:10267000591D483601E0500714F0485651408D016D
:10268000212F220F220B322F0E948F342801390173
:102690008A01212F220F220B322F0E948F34080132
:1026A000190145E35AEF6EE87CE3800191010E9435
:1026B0004F350E94653AA201B3010E944F352801AF
:1026C00039018D01212F220F220B322F0E948F34CE
:1026D000A201B3010E94EE340E949C349C01220F9F
:1026E000331FF901EF51F84D0083118301968830B3
:1026F00000E090070CF4B5CFEAE00C94D6360E94C7
:10270000CA36402E042D10E0000F111FF801E251CF
:10271000F64D20813181042D10E0000F111FF801CA
:10272000E851F64D0081118195DFB1D106E00E949C
:102730003A03E0911B2AF0911C2AF3970CF427C16D
:1027400080E09CE5A1ECB7E400E010E00093312AC2
:102750001093322A08C0E1E3FAE200811181065F9A
:102760001F4F008311830091312A1091322A0836BD
:1027700021E01207BCF52091C7243091C8240091B4
:10278000312A1091322A66DF05E00E943A03009157
:102790001B2A10911C2A212F220F220B322F0E945C
:1027A0008F34AC01BD010E945136A8F600911B2A5E
:1027B00010911C2A212F220F220B322F0E948F34BE
:1027C000C801D9010091312A1091322A00932D2A93
:1027D00010932E2AE0911B2AF0911C2AB8970CF036
:1027E000BACF54C080E09CE5A1ECB7E40AE010E069
:1027F00002D100E010E00093C7241093C82408C061
:10280000E7ECF4E200811181025E1F4F0083118327
:102810000091C7241091C824083E27E01207B4F5A0
:102820002091C7243091C82400912D2A10912E2A7E
:1028300011DF05E00E943A0300911B2A10911C2A27
:10284000212F220F220B322F0E948F34AC01BD01A9
:102850000E945136A8F600911B2A10911C2A212FA4
:10286000220F220B322F0E948F34C801D901009110
:10287000C7241091C82400932F2A1093302AE09186
:102880001B2AF0911C2A74970CF0BACFE0912D2AE4
:10289000F0912E2A3B9744F0EDE2FAE2008111819B
:1028A0000450104000831183E0912F2AF091302AC8
:1028B000759744F0EFE2FAE2008111810F50104069
:1028C0000083118320912F2A3091302A00912D2AE4
:1028D00010912E2ABFDE20912F2A3091302A042D0C
:1028E00010E0000F111FF801E251F64D20833183F3
:1028F00020912D2A30912E2A042D10E0000F111F57
:10290000F801E851F64D20833183042D10E0000FCB
:10291000111FF801E851F64D3181232F042D10E0ED
:10292000000F111F0E5D1F4F0E94630C042D10E05D
:10293000000F111FF801E851F64D2081042D10E021
:10294000000F111F0D5D1F4F0E94630C042D10E03E
:10295000000F111FF801E251F64D3181232F042D94
:1029600010E0000F111F085D1F4F0E94630C042D23
:1029700010E0000F111FF801E251F64D2081042DE7
:1029800010E0000F111F075D1F4F0E94630C0FEF37
:102990000093FB29E5E00C94DB3634E030934009EA
:1029A0003091112A329F00926A0910926B090093AC
:1029B00066091093670908950E94CC36C801A22FBA
:1029C00004E00093400943E00091112A0E947C3307
:1029D000E02FF0E031964A2F50E08F010E949A33A9
:1029E00000936A0910936B098093660990936709B5
:1029F000E3E00C94DD3624E044E650E00E949A3394
:102A0000CCDF0091F42910E0000F111FF801EA5209
:102A1000F64D0081118148E750E00E94C6330E5FF9
:102A20000E943A0300E00093400908958A93812FA1
:102A300010E0E1DF00E41CE91ED0082F10E0DBDF2E
:102A4000899108950E94CB36D80181E090E00CC0B6
:102A500044E050E08C010E94C633202F8D019DDFA1
:102A600000E41CE908D00196843100E0900784F36B
:102A7000E4E00C94DC364091F72950E00E94AE333C
:102A80000150104098018901232BD1F7089526E3C6
:102A900031E201E215E20E94183B00E80E94D802F0
:102AA00000E310E0A8DF08950E94E03240E050E02B
:102AB00064E672E40E944F350E949C3408950E949F
:102AC000E03240E050E064E672E40E944F350E943C
:102AD0009C340B3520E0120714F00BE510E0063AA9
:102AE0002FEF120714F405EA1FEF08950E94C7366E
:102AF000D8018091F42990E001969A938A9327E473
:102B000031E201E215E20E94183B229600E80E94A1
:102B1000D802A13000E0B00714F180E0082F10E0E7
:102B200020E030E00E949A34280139018D01212FE4
:102B3000220F220B322F0E948F340E94E536A8010B
:102B4000B901820193010E94513678F5082F075789
:102B50000E9438020EE30E947C028395DFCF80E062
:102B600008C006E8081B0E9438020CE30E947C02A1
:102B70008395082F10E020E030E00E949A3428016D
:102B800039010FEF1FEFAD010E949A33212F220F61
:102B9000220B322F0E948F340E94E536A801B90122
:102BA000820193010E945136E0F200E315E763DFF2
:102BB000E8E00C94D8369A938A9300E010E080E025
:102BC00090E019C0E0E0F2E02081286020832091AD
:102BD0002B022223E1F321E020932B022091120209
:102BE00030911302020F131F035C1040112312F4E3
:102BF00000E010E00196803A20E092071CF34DE4DB
:102C000050E00E94C633899199910895E0E0F2E086
:102C1000008100610083009133020023E1F301E0B1
:102C20000093330240910B2A50E00091140210915E
:102C300015020E94AE3308950091F42910E0000FB0
:102C4000111FF801E452F64D008111812DDC009135
:102C5000F42910E0000F111FF801E452F64D008135
:102C600011815EDC0091F42910E0000F111FF801C2
:102C7000E452F64D208131810091F42910E0000FDB
:102C8000111FF801EE51F64D208331830091F42994
:102C900010E0000F111FF801EE51F64D0081118177
:102CA000C7DB08950091F42910E0000F111FF8010F
:102CB000E452F64D00811181F7DB0091F42910E018
:102CC000000F111FF801E452F64D0081118128DC3C
:102CD0000091F42910E0000F111FF801EE51F64D9C
:102CE00000811181A5DB08950E94CB36D8010091A7
:102CF000042A002311F088E40DC0BB2312F48CE3F6
:102D000009C04AE050E08D010E94C633102F06E052
:102D1000109F802D00E80E94380290E0FC01E45FE3
:102D2000FC4F04910E947C0201E80E94380290E06E
:102D3000FC01E35FFC4F04910E947C0202E80E94C8
:102D4000380290E0FC01E25FFC4F04910E947C029B
:102D500000EC0E94380290E0FC01E15FFC4F04911E
:102D60000E947C0201EC0E94380290E0FC01E05FCE
:102D7000FC4F04910E947C0202EC0E94380290E019
:102D8000FC01EF5EFC4F04910E947C020091042A3A
:102D9000002311F088E40CC0BB2312F482E408C0C5
:102DA0004AE050E08D010E94C63306E0409F802D2E
:102DB00004E80E94380290E0FC01E45FFC4F0491BB
:102DC0000E947C0205E80E94380290E0FC01E35F6B
:102DD000FC4F04910E947C0206E80E94380290E0B9
:102DE000FC01E25FFC4F04910E947C0204EC0E9413
:102DF000380290E0FC01E15FFC4F04910E947C02EC
:102E000005EC0E94380290E0FC01E05FFC4F049169
:102E10000E947C0206EC0E94380290E0FC01EF5E0A
:102E2000FC4F04910E947C0203E80E94380200E2F9
:102E30000E947C0203EC0E94380200E20E947C02A5
:102E4000E4E00C94DC360E94CB36802F082F10E093
:102E5000000F111FF801EA52F64DA081B1811196C1
:102E6000AD01652F660F660B762F00E01CE62CED9A
:102E700032E00E942D3443E00E94023448E050E0EA
:102E800060E070E00E94DA334EE650E060E070E00F
:102E90000E942D34D80146E450E08D010E94AE33EB
:102EA000009353291093542990E0880F991FFC0137
:102EB000EA52F64D0081118144E150E00E94C63390
:102EC00000935529109356290091F929013029F4CE
:102ED000A0935129B093522906C0AA0FBB1FA093FB
:102EE0005129B0935229E4E00C94DC368A93802F68
:102EF000F89410E500E39ADD8823F1F400E0A3DF05
:102F000001E00093F5290CED15E02091F42930E063
:102F1000220F331FF901E653F64D0083118309E5B3
:102F200013E02091F42930E0220F331FF901E05320
:102F3000F64D008311833FC08130F1F401E083DF5F
:102F400002E00093F52908E513E02091F42930E030
:102F5000220F331FF901E653F64D0083118309E96F
:102F600012E02091F42930E0220F331FF901E053E1
:102F7000F64D008311831FC08230E9F402E063DF65
:102F800002E00093F52907E512E02091F42930E0F2
:102F9000220F331FF901E653F64D008311830AE433
:102FA00011E02091F42930E0220F331FF901E053A2
:102FB000F64D008311830091F42910E0000F111FDA
:102FC000F801EA52F64D0081118100932609109311
:102FD00027094091172A50E00FEF10E00E949A3322
:102FE000DBDA0091F42910E0000F111FF801E25123
:102FF000F64D208131810091F42910E0000F111F5E
:10300000F801E851F64D0081118124DB0091F4298B
:1030100010E0000F111FF801E452F64D00811181FC
:1030200043DA0091F42910E0000F111FF801E45277
:10303000F64D0081118174DA0091F42910E0000F3F
:10304000111FF801EE51F64D00811181F1D98991DE
:1030500008950E94CB36802F082F10E0000F111F1B
:10306000F801EA52F64DA081B1811196AD01652FAC
:10307000660F660B762F00E01CE62CED32E00E9416
:103080002D3443E00E9402341A930A9390E0019693
:103090009A938A9329E531E201E215E20E94183BF6
:1030A000249600E80E94D8022CE631E201E215E203
:1030B0000E94183B00EC0E94D80202E00E943A03F2
:1030C000789400E00093042A01E00093FC290AE0D0
:1030D0000093052A00E010E000934B2910934C293F
:1030E0000093492910934A2901E010E00093252A12
:1030F0001093262A00915529065F0E943A03E4E0C6
:103100000C94DC360E94CC3680914D2990914E294A
:103110000197873500E0900708F059C04AE050E079
:1031200000914729109148290E94C633402F4A5FD9
:103130000091192A10911A2A0E94A83301700023C5
:1031400009F045C00091142A013031F42091002A81
:1031500000E717E122DCA0C00091142A023001F53B
:10316000E0914729F0914829759734F42091002A7D
:1031700000EE1EE212DC90C0009147291091482910
:10318000063420E0120734F02091002A00EA1FE004
:1031900004DC82C02091002A00E717E1FEDB7CC03E
:1031A0002091002AA22F8AE090E04AE050E00091AE
:1031B0004729109148290E94C633801B910B00EDCE
:1031C00017E0AC010E949A332A2FE7DB65C000911B
:1031D000082A002309F460C01091482911230AF03D
:1031E0005BC00091082A10E02091432930914429C6
:1031F000021713070CF050C084E04CEE5FEF009113
:103200004729109148290E94C633801B482F0091FE
:10321000192A10911A2A0E94A83301700023E1F59F
:10322000009147291091482900934B2910934C296C
:1032300042E00091002A0E947C330093002A009112
:10324000472910914829073E2FEF12072CF02091B3
:10325000002A00EB16E3A1DB0091142A0430B9F434
:103260002091002AA22F86E190E04AE050E00091F0
:103270004729109148290E94C633801B910B08EE04
:1032800013E0AC010E949A332A2F87DB05C02091FE
:10329000002A00EC1DE581DBE3E00C94DD360E94A2
:1032A000C336F8940E94DD02E0E8F6E00081086091
:1032B0000083009160060F60009360060091400655
:1032C000006C00934006E0E6F6E0008100620083B7
:1032D000E0E4F6E000810260008300916006006C8B
:1032E0000093600608E10093110608E100931206BE
:1032F00008E10093130608E10093300608E100930B
:10330000520608E1009353060E9403020091F82937
:10331000023011F479D802C00E94E0110FE010E0F1
:103320000E943F0C0F3F11F401E001C000E0E8E013
:10333000F6E0108111FD0CC0E8E0F6E0108112FD0E
:1033400007C0E8E2F6E02081217011E0212701C0EA
:1033500020E0022B002309F4CFC02DE731E201E287
:1033600015E20E94183B00EC0E94D802789409E113
:103370000E943A03F89421E00FE010E00E94630CF1
:1033800023E000E110E00E94630C27EE01E110E071
:103390000E94630C22E002E110E00E94630C2DEE1B
:1033A00003E110E00E94630C21E004E110E00E94C0
:1033B000630C23EF05E110E00E94630C80E049C03C
:1033C00020E0082F10E0000F111F0A5E1F4F0E941F
:1033D000630C2BE0082F10E0000F111F095E1F4F38
:1033E0000E94630C20E0082F10E0000F111F045E04
:1033F0001F4F0E94630C2AE0082F10E0000F111FDE
:10340000035E1F4F0E94630C20E0082F10E0000FA6
:10341000111F0E5D1F4F0E94630C20E0082F10E06B
:10342000000F111F0D5D1F4F0E94630C20E0082F3D
:1034300010E0000F111F085D1F4F0E94630C20E079
:10344000082F10E0000F111F075D1F4F0E94630C33
:103450008395833008F4B4CF22E002E410E00E94A8
:10346000630C28E003E410E00E94630C20E005E414
:1034700010E00E94630C25E00EE410E00E94630C53
:1034800021E001E510E00E94630C21E006E510E078
:103490000E94630C20E00CE410E00E94630C20E02A
:1034A0000DE410E00E94630C24EB0FE410E00E9496
:1034B000630C26E300E510E00E94630C24E007E5BE
:1034C00010E00E94630C24E008E510E00E94630C09
:1034D00021E009E510E00E94630C24E000E610E022
:1034E0000E94630C21E002E510E00E94630C21E0E1
:1034F00001E610E00E94630C80E097C0082F10E006
:10350000000F111F005F1F4F0E943F0CB02FA0E063
:10351000082F10E0000F111F0F5E1F4F0E943F0C7D
:1035200010E0A02BB12B082F10E0000F111FF801A5
:10353000EA52F64DA083B183082F10E0000F111F4F
:103540000A5E1F4F0E943F0CB02FA0E0082F10E032
:10355000000F111F095E1F4F0E943F0C10E0A02BAF
:10356000B12B082F10E0000F111FF801E452F64DA7
:10357000A083B183082F10E0000F111F045E1F4FBE
:103580000E943F0CB02FA0E0082F10E0000F111F89
:10359000035E1F4F0E943F0C10E0A02BB12B082FA1
:1035A00010E0000F111FF801EE51F64DA083B1831A
:1035B000082F10E0000F111F0E5D1F4F0E943F0CDF
:1035C000B02FA0E0082F10E0000F111F0D5D1F4F5E
:1035D0000E943F0C10E0A02BB12B082F10E0000F31
:1035E000111FF801E851F64DA083B183082F10E0B8
:1035F000000F111F085D1F4F0E943F0CB02FA0E06D
:10360000082F10E0000F111F075D1F4F0E943F0C95
:1036100010E0A02BB12B082F10E0000F111FF801B4
:10362000E251F64DA083B1838395833008F466CFD1
:1036300002E410E00E943F0C0093072A03E410E02C
:103640000E943F0C0093082A05E410E00E943F0C02
:1036500000930A2A06E510E00E943F0C0093142A0A
:103660000EE410E00E943F0C0093172A01E510E0E1
:103670000E943F0C0093132A0FE410E00E943F0CBD
:1036800000930C2A00E510E00E943F0C00930B2AE7
:1036900002E510E00E943F0C0093F82907E510E0D6
:1036A0000E943F0C0093112A08E510E00E943F0C95
:1036B0000093122A01E610E00E943F0C0093F929C2
:1036C00009E510E00E943F0C03700093162A00E603
:1036D00010E00E943F0C0093182A0CE410E00E94B6
:1036E0003F0CA02FB0E00DE410E00E943F0C102F23
:1036F00000E0A02BB12BA093192AB0931A2A01E065
:1037000010E80093192A10931A2A08E00093082A57
:1037100004E00093072A01E00093132A0091480671
:103720000C700093F6290091F6290C3021F402E088
:103730000093F4290FC00091F629083021F401E02C
:103740000093F42907C00091F629043019F400E031
:103750000093F4290E9403020091F829023019F421
:103760000E94041202C00E94E01103E200930108CB
:1037700007E00093000806E910E000932608109384
:1037800027080091122A10E000932A0810932B08B2
:1037900007E00093400804ED11E0009366081093E1
:1037A000670801E00093460801E00093000903E088
:1037B000009306090091A20007600093A2000E94F6
:1037C00023030091F42910E0000F111FF801E251CA
:1037D000F64D208131810091F42910E0000F111F76
:1037E000F801E851F64D008111810E942A1304E48A
:1037F00014E000930C0210930D020E94000302E0FB
:10380000009322020E941C030E9415030091F429D8
:103810006DDB03E200934109009164060F7300938E
:1038200064062FE831E201E215E20E94183B00EC49
:103830000E94D80220EA31E201E215E20E94183B20
:1038400000E80E94D80200ED17E0FCD800EA1FE073
:10385000F9D800E41FE1F6D800ED17E0F3D800E056
:103860000093400900E0009340090CE30E943A03F2
:10387000009122250B3469F600912325003549F685
:10388000009124250F3429F600916406006C009302
:10389000640600910C2A10E00659164F00931D2A69
:1038A00010931E2A00912525043509F0B2CF789493
:1038B0000AE00E943A03E8E0F6E0008102FD12C04F
:1038C0000FEF0093022A01E00093012A01E0009328
:1038D000032A10E500E3AAD8E8E0F6E0008102FF41
:1038E000FBCF26C100E00093032A809155298B5F0E
:1038F000C0C028E735E00091F42910E0000F111F47
:10390000F801E851F64D008111810E942A1302E06E
:103910000E943A0348E050E000911B2A10911C2AB3
:103920000E94C6330C5F1F4F0093292A10932A2A46
:103930000091292A10912A2A1A930A9321EB31E245
:1039400001E215E20E94183B229600E80E94D8028C
:1039500022EC31E201E215E20E94183B00EC0E94E9
:10396000D802E8E2F6E0008100FFC3CF0091F4291D
:1039700010E0000F111FF801E251F64D2081318156
:103980000091F42910E0000F111FF801E851F64DE5
:10399000008111810E942A134091172A50E00FEFF5
:1039A00010E00E949A330E94CC1202E00E943A0377
:1039B00002D900932B2A10932C2A0091F42910E0AD
:1039C000000F111FF801EA52F64D408151814F5FFF
:1039D0005F4F652F660F660B762F00E01CE62CED1F
:1039E00032E00E942D3443E00E9402340093292AE1
:1039F00010932A2A00912B2A10912C2A1A930A93A9
:103A00000091292A10912A2A1A930A9323ED31E270
:103A100001E215E20E94183B249600E80E94D802B9
:103A200000911B2A10911C2A1A930A9323EE31E26B
:103A300001E215E20E94183B229600EC0E94D80297
:103A40000091F92910E0000F111FF801E85AFC4F0E
:103A5000059114911A930A932FEE31E201E215E2D7
:103A60000E94183B229609EC0E94D80202E00E94B4
:103A70003A03082F802F8A95002309F072CF01E0C6
:103A80000E94380200E21EE40E943B15E0912B2ABE
:103A9000F0912C2A3597CCF426EF31E201E215E2C1
:103AA0000E94183B00E80E94D80200ED10E00E943E
:103AB000FB1400EB10E00E94FB1400ED10E00E94EC
:103AC000FB1404E10E943A0333C000911B2A1091B9
:103AD0001C2A093522E012075CF127E032E201E2FC
:103AE00015E20E94183B00EC0E94D80200ED10E0A5
:103AF0000E94FB1400EB10E00E94FB1400ED10E0AC
:103B00000E94FB1481E012C000E513EC0E943B15FB
:103B1000E8E0F6E0008102FD08C00091F4290E946F
:103B20007F1310E200E30E94161583958E3160F337
:103B300001E00093FC2900E000930D2A06E00093C9
:103B4000052A00E010E000934B2910934C290093C4
:103B5000492910934A29212F220F220B322FE5E702
:103B6000F9E2008311832283338301E010E00093A4
:103B7000252A1093262A05E00E943A0300E310E06C
:103B80000E94FB1402E00E943A0300E310E00E944E
:103B9000FB1416C00091F629043019F400E00093DC
:103BA000F4290091F429A2D90091F42952DA8394DE
:103BB000082D802E053620F0882400E0009340096F
:103BC0000091022A002309F06AC30091042A00230D
:103BD00009F07DC10091F929033009F478C1E5E6C7
:103BE000F9E20081118122813381E9E8F9E2008361
:103BF000118322833383E9E6F9E200811181228176
:103C00003381E1E9F9E20083118322833383E5E71D
:103C1000F9E2008111810093432910934429009116
:103C2000072A0093092A0091132A033029F00091F2
:103C3000092A0E5F0093092A0091092A10E02091B9
:103C4000432930914429021713070CF0F4C0009166
:103C5000012A002309F0EFC0882400E00093052A20
:103C60000091062A03950093062AEDE8F9E2008107
:103C7000118122813381E9E8F9E240815181628139
:103C80007381401B510B620B730B40835183628322
:103C90007383E5E9F9E20081118122813381E1E951
:103CA000F9E24081518162817381401B510B620BAB
:103CB000730B4083518362837383E9E8F9E20081E7
:103CC000118122813381E9E8F9E2408151816281E9
:103CD00073810E94DA3328013901E1E9F9E20081B8
:103CE000118122813381E1E9F9E2408151816281D0
:103CF00073810E94DA33400E511E621E731E8201D0
:103D000093010E948F340E94333B0E949C3443E015
:103D10000E94A8330093232A1093242A1091242A66
:103D200011234AF422E104EF1EE70E94CD1400E2C1
:103D30001EE40E943B15E1E9F9E200811181228134
:103D400033810E948F34A801B9012A013B01E9E8BF
:103D5000F9E200811181228133810E948F34A20116
:103D6000B3010E945F1500934729109348290091E1
:103D7000432910914429212F220F220B322F0E9418
:103D80008F340E94E5360E949C340093002A0091F3
:103D9000002A1091002A019F800149E050E0209103
:103DA000112A30E0421B530B0E94C6330395009347
:103DB000002A0091272A1091282A20914329309126
:103DC00044290217130704F500914329109144294F
:103DD00000934529109346290091472910914829BD
:103DE00000934D2910934E290091232A1091242AE3
:103DF0000093252A1093262A0091432910914429E3
:103E00000093272A1093282A00914D2910914E29BA
:103E100000934B2910934C2900934729109348296C
:103E20000091192A10911A2A013020E8120709F08E
:103E300036C268D934C200E010E000936A091093DA
:103E40006B09E9E8F9E20081118122813381EDE813
:103E5000F9E20083118322833383E1E9F9E20081EF
:103E6000118122813381E5E9F9E200831183228304
:103E7000338300E010E00093272A1093282A009152
:103E8000192A10911A2A013020E81207B9F000917E
:103E9000062A013098F00091452910914629009397
:103EA00043291093442900E010E000934529109322
:103EB000462928D908EE1DEF0E943B150091052ADE
:103EC00003950093052A00E00093062AE8C10091BB
:103ED000042A002309F0ECC00091F929033009F00D
:103EE000E7C0E5E6F9E20081118122813381E9E84A
:103EF000F9E20083118322833383E9E6F9E200814A
:103F0000118122813381E1E9F9E200831183228367
:103F10003383E5E7F9E2008111810093432910938F
:103F20004429E9E8F9E20081118122813381E9E83D
:103F3000F9E240815181628173810E94DA33280164
:103F40003901E1E9F9E20081118122813381E1E95E
:103F5000F9E240815181628173810E94DA33400E1F
:103F6000511E621E731E820193010E948F340E94B3
:103F7000333B0E949C3445E00E94A8330093232ADF
:103F80001093242A1091242A11234AF422E100E0FC
:103F90001DE70E94CD1400E513EC0E943B1593949D
:103FA000092D902E083020F001E00093FC2999247F
:103FB0000091432910914429212F220F220B322FE7
:103FC0000E948F340E94E5360E949C340093002AA0
:103FD0000091002A1091002A019F0092002A00916E
:103FE000002A10E049E050E02091112A30E0421B05
:103FF000530B0E94C63303950093002AE1E9F9E2CE
:1040000000811181228133810E948F34A801B9017E
:104010002A013B01E9E8F9E2008111812281338123
:104020000E948F34A201B3010E945F1500934B29B7
:1040300010934C290091232A1091242A012B39F442
:1040400042E00091002A0E947C330093002A0091F4
:104050004B2910914C29073E2FEF12073CF020917D
:10406000002A00E717E10E94DC1406C02091002A14
:1040700000E21EE40E94DC140091232A1091242AFD
:104080000093252A1093262AE0914329F091442990
:1040900033970CF404C100914D2910914E290093DF
:1040A0004B2910934C290093472910934829F7C0B6
:1040B00042E050E060E070E0E5E6F9E20081118165
:1040C000228133810E942D34E9E8F9E200831183D3
:1040D0002283338342E050E060E070E0E9E6F9E2F9
:1040E00000811181228133810E942D34E1E9F9E2BE
:1040F000008311832283338342E050E060E070E06C
:10410000E5E7F9E200811181228133810E942D349B
:10411000015010400093432910934429E9E8F9E243
:104120000081118122813381E9E8F9E240815181E6
:10413000628173810E94DA3328013901E1E9F9E2F1
:104140000081118122813381E1E9F9E240815181CD
:10415000628173810E94DA33400E511E621E731E0B
:10416000820193010E948F340E94333B0E949C3451
:1041700045E00E94A8330093232A1093242A00913B
:10418000072A10E020914329309144290217130790
:104190000CF07AC00091012A002309F075C000914B
:1041A000062A03950093062A043631F401E00093B1
:1041B000FC2900E00093062A882400E00093052AE9
:1041C0001091242A11234AF422E100E01DE70E9405
:1041D000CD1400E513EC0E943B150091432910918A
:1041E0004429212F220F220B322F0E948F340E944C
:1041F000E5360E949C340093002A0091002A109119
:10420000002A019F800149E050E02091112A30E00E
:10421000421B530B0E94C6330E5F0093002A00918D
:10422000062A043060F02091002A00EE1EE2409140
:10423000432950914429041B150B0E94CD14009171
:10424000232A1091242A0093252A1093262AE1E993
:10425000F9E200811181228133810E948F34A8010B
:10426000B9012A013B01E9E8F9E2008111812281CB
:1042700033810E948F34A201B3010E945F15009325
:104280004B2910934C290BC000E00093400900E03B
:104290000093062A0091052A03950093052A0091B0
:1042A000052A083C41F010E00091062A083C19F06C
:1042B0001060112399F000E010E000934B29109357
:1042C0004C290093492910934A2900E010E00093FB
:1042D000252A1093262A01E00093FC290091012A47
:1042E000E0E6F3E00C947A3600914B2910914C29CA
:1042F0000093292A10932A2AE091252AF091262A50
:1043000031974CF00091292A10912A2A00934929CB
:1043100010934A2908C00091492910914A29009315
:10432000292A10932A2A0091F829023009F090C016
:104330000091292A10912A2A0E94741604E610E09E
:104340000E943B150091252A1091262A212F220F29
:10435000220B322F0E948F340E94E5360E949C343B
:104360000093292A10932A2A0091052A053048F043
:1043700028E132E201E215E20E94183B07EC0E94BC
:10438000D8020091042A002339F00EE310E00093D4
:104390002B2A10932C2A06C006E010E000932B2A4B
:1043A00010932C2A80E009C0082F08530E9438027D
:1043B00000912B2A0E947C02839590E00091292A8B
:1043C00010912A2A801791077CF30091C92910E0E7
:1043D0001A930A930091132A10E01A930A930091FA
:1043E000072A10E01A930A930091082A10E01A9302
:1043F0000A9322E232E201E215E20E94183B28967B
:1044000007E80E94D8020E94061600932B2A1093F8
:104410002C2A4AE050E000912B2A10912C2A0E946D
:10442000C6335A934A934AE050E000912B2A1091E8
:104430002C2A0E94C6331A930A932DE232E201E23B
:1044400015E20E94183B24960DE80E94D80212C57E
:1044500010912A2A112372F00091292A10912A2AF8
:104460001A930A9324E332E201E215E20E94183B18
:1044700022960DC00091292A10912A2A1A930A9394
:104480002BE332E201E215E20E94183B229600E89B
:104490000E94D8020A2DA02EA394002391F4B09478
:1044A000BB2049F400911B2A10911C2A00932B2A4F
:1044B00010932C2A06C00E94061600932B2A1093F4
:1044C0002C2A0091252A1091262A212F220F220B17
:1044D000322F0E948F340E94E5360E949C34009354
:1044E000292A10932A2A0091292A10912A2A083071
:1044F00020E0120731F40FEF10E00093292A109307
:104500002A2A04E80E9438020091292A0E947C028B
:1045100010912A2A112352F421E432E201E215E239
:104520000E94183B04E80E94D8021EC00091C929CD
:1045300010E01A930A930091132A10E01A930A9339
:104540000091072A10E01A930A930091082A10E0BC
:104550001A930A9323E432E201E215E20E94183B27
:10456000289605E80E94D802BB20E1F04AE050E01E
:1045700000912B2A10912C2A0E94C6335A934A93F9
:104580004AE050E000912B2A10912C2A0E94C63359
:104590001A930A932FE432E201E215E20E94183BDB
:1045A00024960DC000912B2A10912C2A1A930A935D
:1045B00027E532E201E215E20E94183B22960CE860
:1045C0000E94D8020091042A002309F053C00091F0
:1045D000052A053048F02CE631E201E215E20E949E
:1045E000183B00EC0E94D8028091292AE0914729CB
:1045F000F091482931977CF0009147291091482982
:10460000045C1F4F4AE050E00E94C63300934F29DC
:104610001093502912C042E050E0009147291091B8
:1046200048290E94C6330E5C1F4F4AE050E00E94AA
:10463000C63300934F291093502900914F290054FD
:104640000E943802813058F00091052A013020F094
:1046500007E00E947C0203C004E00E947C0205EC9B
:104660000E9438020FE20E947C0200ED17E00E94D7
:104670003B1500C443E00091232A1091242A0E9494
:10468000A8330093292A10932A2A0091292A1091ED
:104690002A2A033C21E0120744F400E030912A2A40
:1046A00033231AF00060002331F002EC11E0009394
:1046B000292A10932A2A2DE532E201E215E20E940E
:1046C000183B00EC0E94D80280E00FC0082F07536F
:1046D0000E9438020EE30E947C0206EC081B0E9436
:1046E00038020CE30E947C028395082F10E020E042
:1046F00030E00E949A34280139010091292A109152
:104700002A2A212F220F220B322F0E948F340E943F
:10471000E536A801B901820193010E945136B0F239
:1047200000ED17E00E943B15A5C300911B2A1091D4
:104730001C2A1A930A932EE632E201E215E20E9445
:10474000183B229600E80E94D80200910C2A10E043
:104750001A930A9320E832E201E215E20E94183B24
:10476000229600EC0E94D80202E00E943A0382C323
:104770000E9406160093292A10932A2A4AE050E044
:104780000091292A10912A2A0E94C6335A934A93EB
:104790004AE050E00091292A10912A2A0E94C6334B
:1047A0001A930A9322E932E201E215E20E94183BD1
:1047B000249600E80E94D80200910B2A10E01A9378
:1047C0000A9326EA32E201E215E20E94183B2296A1
:1047D00000EC0E94D80202E00E943A034BC30E9400
:1047E000DB150093292A10932A2A0091F42910E05E
:1047F000000F111FF801EA52F64D408151814F5FC1
:104800005F4F652F660F660B762F00E01CE62CEDE0
:1048100032E00E942D3443E00E94023400932B2AA0
:1048200010932C2A00915129109152291A930A931E
:104830000091292A10912A2A1A930A93E091F429C7
:10484000F0E03196FA93EA9327EB32E201E215E2C7
:104850000E94183B269600E80E94D80200912B2A5D
:1048600010912C2A1A930A9329EC32E201E215E204
:104870000E94183B229600EC0E94D80200E21EE43F
:104880000E943B15F7C200911B2A10911C2A1A9313
:104890000A93E091F429F0E03196FA93EA9328ED37
:1048A00032E201E215E20E94183B249600E80E94E1
:1048B000D8020091F42910E0000F111FF801E25115
:1048C000F64D008111811A930A9324EE32E201E23F
:1048D00015E20E94183B229609E80E94D8020FEDCB
:1048E00010E01A930A930091F42910E0000F111FB1
:1048F000F801E851F64D008111811A930A930AEAF2
:1049000010E01A930A932DEE32E201E215E20E94C2
:10491000183B269600EC0E94D8020091FB29002348
:1049200021F409E80E94380203C009EC0E94380211
:104930000EE30E947C0200E117E20E943B159AC23E
:1049400040E250E060E070E0E9E6F9E200811181C8
:10495000228133810E942D340E94761521E033E2BA
:1049600001E215E20E94183B00EC0E94D8020FED14
:1049700010E01A930A930091F42910E0000F111F20
:10498000F801E452F64D008111811A930A930AEA64
:1049900010E01A930A932EE033E201E215E20E943E
:1049A000183B26960AEC0E94D80200E117E20E940A
:1049B0003B1560C20FEF0093042A48E050E060E02E
:1049C00070E0E5E7F9E200811181228133810E94E4
:1049D0002D340E94761528E133E201E215E20E94AF
:1049E000183B00EC0E94D8020FED10E01A930A93D6
:1049F0000091F42910E0000F111FF801EE51F64D5F
:104A0000008111811A930A930AEA10E01A930A931B
:104A10002EE033E201E215E20E94183B26960AECF2
:104A20000E94D80200E117E20E943B1523C20091C8
:104A3000112A10E01A930A9324E233E201E215E20C
:104A40000E94183B229600E80E94D8022CE233E232
:104A500001E215E20E94183B06E80E94D80227E313
:104A600033E201E215E20E94183B00EC0E94D802FA
:104A700080E010C0082F0A530E943802082F0E94BD
:104A80007C02883031F40EEC0E9438020FEF0E9455
:104A90007C0283950091112A081760F702E00E94BA
:104AA0003A03E8C10091142A033039F40AE010E017
:104AB0000093292A10932A2A14C00091142A043042
:104AC00039F40EE010E00093292A10932A2A09C035
:104AD0000091142A10E0000F111F0093292A10934F
:104AE0002A2A0091292A10912A2A1A930A9328E443
:104AF00033E201E215E20E94183B229600E80E9490
:104B0000D8022CE233E201E215E20E94183B06E8EB
:104B10000E94D80220E533E201E215E20E94183B30
:104B200000EC0E94D80280E010C0082F0A530E94B7
:104B30003802082F0E947C02883031F40EEC0E946B
:104B400038020FEF0E947C0283950091142A081707
:104B500060F702E00E943A038DC10091F82910E04D
:104B60001A930A9321E633E201E215E20E94183B10
:104B7000229600E80E94D80223E733E201E215E220
:104B80000E94183B00EC0E94D80280E010C0082F61
:104B90000A530E943802082F0E947C02883031F4A8
:104BA0000EEC0E9438020FEF0E947C028395009168
:104BB000F829081760F702E00E943A035BC10091F0
:104BC000F92910E0000F111FF801E85AFC4F059178
:104BD00014911A930A9325E833E201E215E20E9448
:104BE000183B229600E80E94D80223E933E201E252
:104BF00015E20E94183B00EC0E94D80280E010C031
:104C0000082F0A530E943802082F0E947C02883025
:104C100031F40EEC0E9438020FEF0E947C02839563
:104C20000091F929081760F702E00E943A0322C1B7
:104C30000091122A10E01A930A9325EA33E201E266
:104C400015E20E94183B229600E80E94D80227EB4A
:104C500033E201E215E20E94183B00EC0E94D80208
:104C600080E010C0082F0A530E943802082F0E94CB
:104C70007C02883031F40EEC0E9438020FEF0E9463
:104C80007C0283950091122A081760F703E00E94C6
:104C90003A03F0C00E94DB151A930A9329EC33E221
:104CA00001E215E20E94183B229600E80E94D80219
:104CB0002CE233E201E215E20E94183B06E80E9472
:104CC000D80220ED33E201E215E20E94183B00EC2D
:104CD0000E94D80280E010C0082F0A530E943802B8
:104CE000082F0E947C02883031F40EEC0E943802BA
:104CF0000FEF0E947C0283950091172A081760F736
:104D000002E00E943A03B6C000911B2A10911C2AAF
:104D10001A930A9321EE33E201E215E20E94183B56
:104D2000229600E80E94D8022CE233E201E215E26A
:104D30000E94183B06E80E94D80228EE33E201E206
:104D400015E20E94183B00EC0E94D80280E010C0DF
:104D5000082F0A530E943802082F0E947C028830D4
:104D600031F40EEC0E9438020FEF0E947C02839512
:104D70000091162A081760F702E00E943A037AC0F1
:104D80000091182A10E01A930A9329EF33E201E206
:104D900015E20E94183B229600E80E94D8022CE2FD
:104DA00033E201E215E20E94183B06E80E94D802B5
:104DB00020E034E201E215E20E94183B00EC0E9480
:104DC000D80280E010C0082F0A530E943802082F32
:104DD0000E947C02883031F40EEC0E9438020FEF02
:104DE0000E947C0283950091182A081760F702E060
:104DF0000E943A0301E00093FE293CC00091FE2985
:104E00000023C1F121E134E201E215E20E94183BE6
:104E100000E80E94D80280E004C000E20E947C0208
:104E20008395803190F4082F00540E943802482F57
:104E30000091192A10911A2A0E94A83301700023A8
:104E400061F303E20E947C02EBCF05EC0E94380282
:104E50000FE20E947C0200910D2A00540E94380249
:104E60000EE00E94380200E00093FE2908EE1DEFDC
:104E70000E943B1590E0E8E0F6E0008103FD9BC056
:104E800000E00093400901E00093FC29E8E0F6E02F
:104E9000008103FD51C008EE1DEF0E943B15939564
:104EA000092F902F209155293091562910E0201775
:104EB000310760F70091022A00950093022A0091C1
:104EC000F829023011F40E94041201E00E94380215
:104ED0000091022A002381F400E00093012A40910E
:104EE000172A50E00FEF10E00E949A330E94CC1274
:104EF00003E00E943A030CC007E00093012A03E09C
:104F00000E943A0300E010E00E94CC120E94E011DF
:104F100001E00093FE2900E00093032A00E00093E3
:104F2000042A0AE510E00E94FB1401E00093FC292A
:104F300002E00E943A038BC10091022A002349F447
:104F40000091042A00950093042A0AEA0093052A96
:104F500029C00CE00E9438020091032A013059F464
:104F60000091012A03950093012A073070F001E0B7
:104F70000093012A0AC00091012A03950093012A97
:104F8000003118F007E00093012A0091012A0C304B
:104F900049F44091172A50E00FEF10E00E949A3335
:104FA0000E94CC1208E210E00E94FB1405E00E946F
:104FB0003A030C948F32E8E2F6E0008100FD5BC416
:104FC00000E0009340090091012A005081F00A9509
:104FD00009F448C1025009F4A6C10A9509F4C4C3F2
:104FE0000A9509F435C20A5009F4ECC33CC4E8E25E
:104FF000F6E0008100FDFFC008EE1DEF0E943B15AA
:105000009395092F902F209155293091562910E022
:105010002017310760F700E310E00E94FB14E1E77E
:10502000F9E200811181228133810E948F34A8012D
:10503000B9012A013B01EDE6F9E2008111812281EB
:1050400033810E948F34A201B3010E945F15009347
:105050004729109348290091232A1091242A212FAF
:10506000220F220B322F0E948F340E94E53640918E
:105070004729509148295A934A9340E050E060E014
:1050800070E40E944F350E949C341A930A9322E2E6
:1050900034E201E215E20E94183B249600E80E94E7
:1050A000D8020091472910914829053C2FEF12079B
:1050B00064F400E02091472930914829253A1FEFF8
:1050C00031071CF00060002399F027E334E201E28D
:1050D00015E20E94183B00EC0E94D80200EB10E0A1
:1050E0000E94FB14E8E2F6E0008100FFFBCFAFC0B6
:1050F00028E434E201E215E20E94183B00EC0E9431
:10510000D80200E210E00E94FB140091F42910E0A4
:10511000000F111FF801E452F64D0081118120911A
:10512000472930914829021B130B0A5510400F5F85
:105130001F4F2091F42930E0220F331FF901EE5167
:10514000F64D008311830091F42910E0000F111F28
:10515000F801EE51F64D1181112372F40091F429FA
:1051600010E0000F111FF801EE51F64D0081118182
:1051700008591E4F008311830E945216E8E2F6E0A0
:10518000008100FFFBCF01E00093FC292CE631E217
:1051900001E215E20E94183B00EC0E94D802009147
:1051A000F42910E0000F111FF801EE51F64D318186
:1051B000232F0091F42910E0000F111F045E1F4FF0
:1051C0000E94630C0091F42910E0000F111FF801F8
:1051D000EE51F64D20810091F42910E0000F111FCF
:1051E000035E1F4F0E94630C05E00E943A0301E03A
:1051F0000093FC292CC001E00093FC2900911B2A9C
:1052000010911C2A1A930A9329E534E201E215E26F
:105210000E94183B229600E80E94D8022CE631E258
:1052200001E215E20E94183B00EC0E94D80200E364
:1052300010E00E94FB140091062A002311F401E003
:1052400001C000E00093052A0AE00E943A032BE621
:1052500034E201E215E20E94183B00E80E94D80205
:105260000C948F3200E010E00E94CC120E9447158F
:1052700008E813E100932B2A10932C2A00E010E099
:105280000093292A10932A2A31C00091292A1091CB
:105290002A2A0659164F00931D2A10931E2A00E64B
:1052A0001AEE0E943B1500E61AEE0E943B15009193
:1052B0001B2A10911C2A20912B2A30912C2A02178C
:1052C000130764F400911B2A10911C2A00932B2AC7
:1052D00010932C2A0091292A00930C2AE9E2FAE281
:1052E000008111810E5F1F4F008311830091292AD5
:1052F00010912A2A0B3F20E012073CF220910C2A41
:105300000FE410E00E94630C10E600E40E94161502
:105310004091172A50E00FEF10E00E949A330E944C
:10532000CC120C948F32A0E0B0E00E94471500919F
:10533000F42910E0000F111FF801E053F64D008131
:1053400011810093292A10932A2A27C00091292A23
:1053500010912A2A009326091093270903E00E943E
:105360003A030E94DB15A017B1077CF4D801209105
:10537000292A30912A2A0091F42910E0000F111FE8
:10538000F801EA52F64D20833183E9E2FAE2008126
:1053900011810C5F1F4F008311832091292A3091C6
:1053A0002A2A0091F42910E0000F111FF801E6539A
:1053B000F64D008111812017310744F20091F42944
:1053C00010E0000F111FF801EA52F64D0081118123
:1053D000009326091093270910E400E50E94161592
:1053E0000091F42910E0000F111FF801EA52F64D68
:1053F0003181232F0091F42910E0000F111F005F6D
:105400001F4F0E94630C0091F42910E0000F111F40
:10541000F801EA52F64D20810091F42910E0000FC6
:10542000111F0F5E1F4F0E94630C0C948F3223E9F3
:1054300034E201E215E20E94183B00E80E94D80223
:1054400000E810E00E94FB1400E810E00E94FB144A
:10545000E8E2F6E0008100FD71C100E61AEE0E946C
:105460003B159395092F902F20915529309156295E
:1054700010E02017310760F701E00093FF2921E7D2
:1054800034E201E215E20E94183B00E80E94D802D3
:1054900000E310E00E94FB1401E00093FC2900915E
:1054A0005529065F0E943A0322E834E201E215E240
:1054B0000E94183B00E80E94D80200E310E00E941E
:1054C000FB1404E10E943A0300E010E00093292A53
:1054D00010932A2A80E029C0E1E7F9E200811181D6
:1054E000228133810E948F34A801B9012A013B0136
:1054F000EDE6F9E200811181228133810E948F342F
:10550000A201B3010E945415E9E2FAE2208131813F
:10551000200F311F20833183009155291091562986
:10552000169507950E943A0383958A30A8F24AE0BF
:1055300050E00091292A10912A2A0E94C633009334
:10554000292A10932A2A0091F42910E0000F111F34
:10555000F801E452F64D008111810A551040209166
:10556000292A30912A2A021B130B2091F42930E0BA
:10557000220F331FF901E452F64D0083118300918D
:10558000F42910E0000F111FF801E452F64D0081DC
:105590001181093621E0120774F00091F42910E01E
:1055A000000F111FF801E452F64D008111810856D9
:1055B0001140008311830091F42910E0000F111FA6
:1055C000F801E452F64D1181112372F40091F4298F
:1055D00010E0000F111FF801E452F64D0081118117
:1055E00008591E4F008311830E941C1600915529F3
:1055F0000E943A03E1E7F9E20081118122813381BF
:105600000E948F34A801B9012A013B01EDE6F9E2BD
:1056100000811181228133810E948F34A201B30164
:105620000E94541500932B2A10932C2A00912B2AA8
:1056300010912C2A0C3A2FEF12070CF0F8CE24EA26
:1056400034E201E215E20E94183B00E80E94D80211
:1056500005E210E00E94FB1405E00E943A0305E217
:1056600010E00E94FB140091F42910E0000F111FBC
:10567000F801E452F64D208131810091F42910E0C7
:10568000000F111FF801EE51F64D20833183009178
:10569000F42910E0000F111FF801EE51F64D0081C2
:1056A00011810E9418120091F42910E0000F111FBF
:1056B000F801E452F64D3181232F0091F42910E0D6
:1056C000000F111F0A5E1F4F0E94630C0091F42906
:1056D00010E0000F111FF801E452F64D20810091F7
:1056E000F42910E0000F111F095E1F4F0E94630C88
:1056F0000091F42910E0000F111FF801EE51F64D52
:105700003181232F0091F42910E0000F111F045E56
:105710001F4F0E94630C0091F42910E0000F111F2D
:10572000F801EE51F64D20810091F42910E0000FB0
:10573000111F035E1F4F0E94630C8ACE0091FF2948
:10574000002389F425EB34E201E215E20E94183BC4
:1057500000E80E94D80208EE1DEF0E943B1500E50C
:1057600010E00E94FB14DBC6E8E2F6E0008100FDD9
:105770001CC008EE1DEF0E943B159395092F902F3A
:10578000209155293091562910E02017310760F7F4
:1057900000E610E00E94FB140091F4290E947F13A0
:1057A00010E200E30E94161552CD0091FB290095EE
:1057B0000093FB2902E310E00E94FB1404E00E9426
:1057C0003A03ADC601E010E00093292A10932A2A7B
:1057D00040910D2A0091292A10912A2A0E94A23371
:1057E0000093292A10932A2A40910D2A0091192A00
:1057F00010911A2A0E94A8330170002399F0009199
:10580000292A10912A2A00951095E9E1FAE22081CF
:105810003181202331232083318310E500E40E946D
:10582000161510C00091292A10912A2AE9E1FAE2FE
:1058300020813181202B312B2083318310E300E440
:105840000E94161501E00093FE292091192A0CE40C
:1058500010E00E94630C30911A2A232F0DE410E00F
:105860000E94630C5CC601E00093FC2908E210E092
:105870000E94FB1454C6E8E0F6E0008102FD1BC361
:1058800000E0009340090091012AE6E8F3E00C945F
:105890007A36E8E0F6E0008102FD26C008EE1DEF52
:1058A0000E943B158395082F802F20915529309118
:1058B000562910E02017310760F700910A2A009559
:1058C00000930A2A20910A2A05E410E00E94630C42
:1058D00001E00093FF2900E510E00E94FB1400E6C0
:1058E0001AEE0E943B151EC60091FF29002381F489
:1058F0000091072A03950093072A0A3018F000E068
:105900000093072A2091072A02E410E00E94630C0A
:10591000CAC200910C2A039500930C2A0B3F18F081
:1059200000E000930C2A20910C2A0FE410E00E9462
:10593000630C00E41CE90E943B15B5C200910B2AE0
:10594000039500930B2A0D3318F001E000930B2A06
:1059500020910B2A00E510E00E94630C00E41CE992
:105960000E943B15A0C20091F42910E0000F111F06
:10597000F801EA52F64D008111810150104020914A
:10598000F42930E0220F331FF901EA52F64D00836B
:1059900011832091F42930E0220F331FF901E053E5
:1059A000F64D2081318102171307A4F40091F429E8
:1059B00010E0000F111FF801E053F64D20813181F6
:1059C0000091F42910E0000F111FF801EA52F64D82
:1059D000208331830091F42910E0000F111FF8019A
:1059E000EA52F64D00811181009326091093270990
:1059F0000091F4290E9423170091F42910E0000F70
:105A0000111FF801EA52F64D3181232F0091F4293C
:105A100010E0000F111F005F1F4F0E94630C0091E8
:105A2000F42910E0000F111FF801EA52F64D208111
:105A30000091F42910E0000F111F0F5E1F4F0E940C
:105A4000630C31C2E8E0F6E0008101FD1DC020E0FA
:105A500030E00091F42910E0000F111FF801E2512D
:105A6000F64D208331830091F42910E0000F111FBF
:105A7000F801E851F64D2083318304E610E00E94DE
:105A8000FB1406E00E943A030091FB29002309F071
:105A900042C00091F42910E0000F111FF801E251FB
:105AA000F64D008111810F5F1F4F2091F42930E0E6
:105AB000220F331FF901E251F64D008311830130AB
:105AC00028E0120764F000E018E02091F42930E0AB
:105AD000220F331FF901E251F64D0083118300912B
:105AE000F42910E0000F111FF801E251F64D318149
:105AF000232F08E210E00E94630C0091F42910E0CB
:105B0000000F111FF801E251F64D208109E210E06B
:105B10000E94630C4BC00091F42910E0000F111F8C
:105B2000F801E851F64D008111810F5F1F4F209160
:105B3000F42930E0220F331FF901E851F64D0083BC
:105B40001183093621E0120764F000E010E0209193
:105B5000F42930E0220F331FF901E851F64D00839C
:105B600011830091F42910E0000F111FF801E85192
:105B7000F64D3181232F0091F42910E0000F111F01
:105B80000E5D1F4F0E94630C0091F42910E0000F7E
:105B9000111FF801E851F64D20810091F42910E021
:105BA000000F111F0D5D1F4F0E94630C0091F4291F
:105BB00010E0000F111FF801E251F64D20813181F4
:105BC0000091F42910E0000F111FF801E851F64D83
:105BD000008111810E942A1302E00E943A0363C1EE
:105BE0000091F42910E0000F111FF801E452F64D66
:105BF000008111810F5F1F4F2091F42930E0220FA7
:105C0000331FF901E452F64D00831183083621E079
:105C1000120764F000E010E02091F42930E0220F38
:105C2000331FF901E452F64D008311830E941C16C4
:105C30000091F42910E0000F111FF801E452F64D15
:105C4000208131810091F42910E0000F111FF8012B
:105C5000EE51F64D208331830091F42910E0000FBE
:105C6000111FF801E452F64D3181232F0091F429E0
:105C700010E0000F111F0A5E1F4F0E94630C00917D
:105C8000F42910E0000F111FF801E452F64D2081B5
:105C90000091F42910E0000F111F095E1F4F0E94B0
:105CA000630C01C10091F42910E0000F111FF801ED
:105CB000EE51F64D008111810F5F1F4F2091F429A5
:105CC00030E0220F331FF901EE51F64D00831183AE
:105CD000083621E0120764F000E010E02091F4297A
:105CE00030E0220F331FF901EE51F64D008311838E
:105CF0000091F42910E0000F111FF801EE51F64D4C
:105D0000008111810E9418120091F42910E0000F07
:105D1000111FF801EE51F64D3181232F0CE110E0F7
:105D20000E94630C0091F42910E0000F111FF8018C
:105D3000EE51F64D20810DE110E00E94630CB3C0DE
:105D40000091112A03950093112A093018F008E0F8
:105D50000093112A2091112A07E510E00E94630C9C
:105D6000A2C00091142A03950093142A053018F05C
:105D700004E00093142A2091142A06E510E00E9402
:105D8000630C91C00091F82903950093F829033022
:105D900018F002E00093F8292091F82902E510E0BC
:105DA0000E94630C80C00091F92903950093F929A2
:105DB000043018F003E00093F9292091F92901E655
:105DC00010E00E94630C01E00093FC290091F4298B
:105DD0000E94231768C00091122A03950093122A8B
:105DE000093018F008E00093122A0BE910E0009344
:105DF0002608109327082091122A08E510E00E9437
:105E0000630CE091122AF0E03196E0932A08F093B7
:105E10002B0849C00091172A03950093172A0930CF
:105E200018F008E00093172A4091172A50E00FEF6E
:105E300010E00E949A330E94CC122091172A0EE49F
:105E400010E00E94630C2FC00091162A0395009366
:105E5000162A043018F003E00093162A2091162A1F
:105E600009E510E00E94630C1EC00091182A0395FA
:105E70000093182A093018F008E00093182A20919E
:105E8000182A00E610E00E94630C0DC000910D2A54
:105E9000039500930D2A003118F000E000930D2ABD
:105EA00001E00093FE2908E210E00E94FB1401E0EB
:105EB0000093FC2934C3E8E0F6E0008101FD2FC324
:105EC00000E0009340090091012AECEAF3E00C9411
:105ED0007A36E8E0F6E0008101FD2BC008EE1DEF08
:105EE0000E943B158395082F802F209155293091D2
:105EF000562910E02017310760F70091132A039507
:105F00000093132A043018F001E00093132A209123
:105F1000132A01E510E00E94630C01E00093FF29C1
:105F200000E510E00E94FB1400E61AEE0E943B150B
:105F3000F9C20091FF29002381F40091082A0395FA
:105F40000093082A0A3018F000E00093082A2091F4
:105F5000082A03E410E00E94630CDAC200910C2AC4
:105F60000A9500930C2A0E3F18F00AEF00930C2AB2
:105F700020910C2A0FE410E00E94630C00E41CE95D
:105F80000E943B15C5C200910B2A0A9500930B2A6B
:105F9000002319F40CE300930B2A20910B2A00E54F
:105FA00010E00E94630C00E41CE90E943B15B0C2A3
:105FB0000091F42910E0000F111FF801EA52F64D8C
:105FC000008111810F5F1F4F2091F42930E0220FD3
:105FD000331FF901EA52F64D008311832091F42911
:105FE00030E0220F331FF901E653F64D2081318155
:105FF00020173107A4F40091F42910E0000F111FBD
:10600000F801E653F64D208131810091F42910E02A
:10601000000F111FF801EA52F64D208331830091E1
:10602000F42910E0000F111FF801EA52F64D00812B
:10603000118100932609109327090091F4290E94E9
:1060400023170091F42910E0000F111FF801EA5204
:10605000F64D3181232F0091F42910E0000F111F1C
:10606000005F1F4F0E94630C0091F42910E0000FA5
:10607000111FF801EA52F64D20810091F42910E039
:10608000000F111F0F5E1F4F0E94630C41C2E8E01A
:10609000F6E0008102FD1DC020E030E00091F4290F
:1060A00010E0000F111FF801E251F64D20833183FB
:1060B0000091F42910E0000F111FF801E851F64D8E
:1060C0002083318304E610E00E94FB1406E00E9466
:1060D0003A030091FB29002309F04AC00091F429FA
:1060E00010E0000F111FF801E251F64D00811181FF
:1060F000015010402091F42930E0220F331FF901A4
:10610000E251F64D00831183112362F400E010E0A8
:106110002091F42930E0220F331FF901E251F64DAE
:10612000008311830091F42910E0000F111FF80182
:10613000E251F64D3181232F0091F42910E0000F38
:10614000111F085D1F4F0E94630C0091F42910E09D
:10615000000F111FF801E251F64D20810091F42942
:1061600010E0000F111F075D1F4F0E94630C49C014
:106170000091F42910E0000F111FF801E851F64DCD
:1061800000811181015010402091F42930E0220F4C
:10619000331FF901E851F64D00831183112362F496
:1061A00008E611E02091F42930E0220F331FF901B5
:1061B000E851F64D008311830091F42910E0000F9F
:1061C000111FF801E851F64D3181232F0091F42978
:1061D00010E0000F111F0E5D1F4F0E94630C009115
:1061E000F42910E0000F111FF801E851F64D20814D
:1061F0000091F42910E0000F111F0D5D1F4F0E9448
:10620000630C0091F42910E0000F111FF801E25116
:10621000F64D208131810091F42910E0000F111F0B
:10622000F801E851F64D008111810E942A1302E025
:106230000E943A036DC10091F42910E0000F111F74
:10624000F801E452F64D0081118101501040209177
:10625000F42930E0220F331FF901E452F64D008398
:106260001183112362F408E611E02091F42930E053
:10627000220F331FF901E452F64D008311830E946F
:106280001C160091F42910E0000F111FF801E452D0
:10629000F64D208131810091F42910E0000F111F8B
:1062A000F801EE51F64D208331830091F42910E07E
:1062B000000F111FF801E452F64D3181232F009198
:1062C000F42910E0000F111F0A5E1F4F0E94630C9B
:1062D0000091F42910E0000F111FF801E452F64D6F
:1062E00020810091F42910E0000F111F095E1F4F5B
:1062F0000E94630C0DC10091F42910E0000F111FE2
:10630000F801EE51F64D00811181015010402091AD
:10631000F42930E0220F331FF901EE51F64D0083CE
:106320001183112362F408E611E02091F42930E092
:10633000220F331FF901EE51F64D008311830091B6
:10634000F42910E0000F111FF801EE51F64D008105
:1063500011810E9418120091F42910E0000F111F02
:10636000F801EE51F64D3181232F0091F42910E010
:10637000000F111F045E1F4F0E94630C0091F4294F
:1063800010E0000F111FF801EE51F64D2081009131
:10639000F42910E0000F111F035E1F4F0E94630CD1
:1063A000B7C00091112A0A950093112A0F3F19F4E2
:1063B00000E00093112A2091112A07E510E00E94C5
:1063C000630CA6C00091142A0A950093142A013088
:1063D00018F401E00093142A2091142A06E510E035
:1063E0000E94630C95C00091F8290A950093F82942
:1063F000013018F401E00093F8292091F82902E512
:1064000010E00E94630C84C00091F9290A95009362
:10641000F929013018F401E00093F9292091F929B4
:1064200001E610E00E94630C01E00093FC2900915A
:10643000F4290E9423176CC00091122A0A95009338
:10644000122A0F3F19F400E00093122A0091122A39
:10645000002331F400E010E0009326081093270891
:106460002091122A08E510E00E94630CE091122AA4
:10647000F0E03196E0932A08F0932B0849C0009190
:10648000172A0A950093172A0F3F19F400E000938A
:10649000172A4091172A50E00FEF10E00E949A331C
:1064A0000E94CC122091172A0EE410E00E94630C87
:1064B0002FC00091162A0A950093162A013018F46D
:1064C00001E00093162A2091162A09E510E00E94A7
:1064D000630C1EC00091182A0A950093182A0F3FDA
:1064E00019F400E00093182A2091182A00E610E021
:1064F0000E94630C0DC000910D2A0A9500930D2A8D
:106500000F3F19F40FE000930D2A01E00093FE29DC
:1065100008E210E00E94FB1401E00093FC2900E077
:106520000093FF2900910C2A10E00659164F0093A2
:106530001D2A10931E2A00910A2A002349F0009177
:1065400064060F73009364060AE20093C92908C029
:1065500000916406006C0093640600E20093C92970
:106560000091480610E00C7010700093292A1093D7
:106570002A2A0091F62910E02091292A30912A2A0E
:106580000217130711F40C94D71D0091292A0093C8
:10659000F6290091F6290C3029F402E00093F42941
:1065A0000C94D11D0091F629083011F00C94CA1DED
:1065B00001E00093F4290C94D11D00008895FECFD2
:1065C0000E94C736C801D9012A013B015CD057D0CF
:1065D00071F48201930153D051F401E2E3E3FAE252
:1065E000008341830FEF1FEF2FE73FE73DC044D00B
:1065F000A201B3010E94EE34AC01BD0140D061F4B0
:1066000042D03AD00E9469360BED1FE029EC10F41D
:106610003FE32AC03FEB28C0A201B3012DD00E9466
:10662000C835080119012FD0820193010E9451360B
:1066300023D0A0F41CD050F424D0A801B9010BED54
:106640001FE029E430E40E9432350EC01AD04BED31
:106650005FE069E470EC0E94EE3406C008D010F4EC
:1066600010D002C00ED03058E8E00C94D8360E940A
:1066700069368001910108958C019D0108950C9463
:1066800047360C94C93940E050E060E070E008956E
:106690003F7741E00C94683A03E20DBF01E20EBF80
:1066A000C0E0D1E20E946837002311F00E944B3A0B
:1066B0000E944F190E94DD320C94DD320D01DA0187
:1066C00040E050E060E070E00E94473639F400E0BE
:1066D00010E04D934C9320E030E00CC0B901660F00
:1066E000771F7E57572F550F550B7D935C932F7750
:1066F00030783F63D00108950024E8E0EA9532F055
:10670000001F001C0416D0F3041AF8CF001F402D00
:1067100000950895FF27442312F4F160419500236A
:1067200012F4F09501950E947C33F0FD0195F1FD86
:1067300041950895149F102D059F100D049F002D65
:10674000110D08954A951AF0000F111FFBCF0895FF
:106750004A951AF015950795FBCF0895002411244A
:10676000EFE0001F111F001C111C0416150610F08D
:10677000041A150AEA95AAF7001F111FA001009537
:10678000109508955195419550400895FF27552340
:1067900012F4F160F7DF112312F4F09507D00E9494
:1067A000AE33F0FD03D0F1FDEDCF089511950195C5
:1067B000104008952224349F302D259F300D169FC0
:1067C000300D079F300D249F202D310D159F200D7A
:1067D000311D069F200D311D149F102D210D321DDE
:1067E000059F100D211D321D049F002D110D221D2E
:1067F000321D08954A952AF03695279517950795E5
:10680000F9CF08954A952AF035952795179507955C
:10681000F9CF0895002411241001E0E2EA9592F0E6
:10682000001F111F221F331F001C111C221C331CB0
:10683000041615062606370688F3041A150A260AD2
:10684000370AECCF001F111F221F331FA001B10117
:1068500000951095209530950895FF27772312F421
:10686000F16015D0332312F4F09509D00E940A3458
:10687000F69508F404D0F69508F409C0089530950B
:106880002095109501951F4F2F4F3F4F08957095FC
:106890006095509541955F4F6F4F7F4F0895FF274B
:1068A000112477FB660F771F089409F4771F67950B
:1068B00017F8EE27002437FB220F331F089409F442
:1068C000331F279507F8089527FD0EC0EE0F001F10
:1068D000111F221F3A953230B8F7332319F427FDE0
:1068E00031E002C027FF30E0E03821F400FF0894D7
:1068F0000EF488940F4F1F4F2F4F3F4F323038F414
:10690000332319F427FD31E002C027FF30E03F3F79
:1069100029F0220F000C379527950895ACC0032E5F
:10692000002012F40E943F34E02F012F122F232F5A
:106930003EE9D1CF0024F8CFBCDF432F4F5748F0BA
:106940004F3148F007FC91C03FE72FEF1FEF0FEFEB
:10695000089533278CC0322F212F102F0E2F4F5127
:1069600041950E94FA3307FE08950C943F34F901D3
:10697000EE0FFF1F37FBFF3F31F0EF2BE12BE02B3A
:106980008894B8940895E02BE12B21F00894989412
:10699000B89408959894889438940895FB01EE0F64
:1069A000FF1F77FBFF3F31F0EF2BE52BE42B8894A3
:1069B000B8940895E42BE52B69F3E8CFEFDF68F096
:1069C00021F43723262F8A010895372FFBCFE6DFE6
:1069D00020F00BF008957327EAF751C0C8DFE8F301
:1069E000B3F361F3DBDFC8F383F3A1F358DF4017A0
:1069F00051076207730731F4011411F10024E89480
:106A000088942BC078F0332E372F732D322E262FFB
:106A1000632D312E152F532D302E042F432D302C66
:106A2000012C132C371739F0669557954795F79534
:106A3000E0407395F7CFE7FBEE0FE0E010246AF03B
:106A4000EF0F041F151F261F60F427951795079554
:106A5000E79508F4689433953ECFEF0B040B150BC4
:106A6000260B39CFE0E87E27B9CF302D30782227AA
:106A70001127002708953FE7302920E8F9CF3FEF9D
:106A80002FEFF6CF8BDFD8F3D1F370783727089547
:106A900085DFA8F3A3F3F9CF3078372793CF67DFEB
:106AA00070F383F3A9F37ADF50F3B3F3A9F3F7DEBE
:106AB0000124E8943F57E040370FEF1F12F0D9F65A
:106AC00003C03A3E90F26894E0E00A92AA933A93A7
:106AD000AA27332422243327049FF001059FF00DB9
:106AE000712D731F149FF00D711D221C069F700DD8
:106AF000211C331C159F700D211C331E249F700D0B
:106B0000211C331E169F200C311CAA1F259F200C10
:106B1000311CA31F269F300CA11D39915EF43395C3
:106B2000A695379427947795F795E7953395313067
:106B3000BCF316C0AA2322F0332351F4339510C0BE
:106B4000339571F4A991099096CFA7FD09C03A95A4
:106B5000EE0FFF1F771F221C331CAA1F3230A8F72D
:106B6000E894FE2B09F068942A2F8101E72FA99160
:106B70000990BACE13DF10F00BF087CF80CF0EDF75
:106B8000E9F3E0F3032E072670CF032E072673CF19
:106B9000EEDEA0F37BF399F301DF80F39BF3A9F31F
:106BA0007EDE012427FD06C0000F111F221F315079
:106BB000E040F8CF67FD06C0440F551F661F7150B7
:106BC000F040F8CFE894371BEF0B3158EF4F2AF025
:106BD000EE23E9F63F3FD9F203C03A3EA8F26894AB
:106BE000E0E0F0E01124139440175107620738F0F9
:106BF000315008F46894000F111F221FEE1F041B70
:106C0000150B260BEF0B000F111F221FEE1F0A9210
:106C100079E17A95AAF0041715072607EF0730F0F7
:106C2000041B150B260BEF0B089401C08894111C54
:106C3000221C331C001C000F111F221FEE1FE9CF66
:106C4000F0F9E894E22BE12BE02B09F0689406942C
:106C5000379427941794E79508F468947395B9F3DB
:106C60000990332311F0F0FF09C03694279417944C
:106C7000E79508F4689433953130BCF3012D122D5B
:106C8000232D32CE8BCE98940895189408956FDEFC
:106C9000D0F3C1F383DEB8F30417150726073707CF
:106CA00008957CDEA0F063DE90F029F0E32FE72763
:106CB0003AF47317089572DE51F04EF00894089577
:106CC000041715072607370719F016F4B8F7889444
:106CD000089564DEE0F34BDED0F3E7DFC0F3089401
:106CE00008957591659155914591159011FA2590EA
:106CF00035900895F9DF041B10E003C0F4DF041B96
:106D0000150B20E030E005C0ECDF041B150B260B53
:106D1000370BB8F010FC17C045910590E00FF11F3C
:106D20000417100540E02407340758F436F40491A2
:106D30000024F101E01BF0090994E00FF11F2590F8
:106D40003590F101099411F4D6F7F1CF31960EF098
:106D5000319650E060E070E045914B3F48F089F398
:106D60004F3F29F04E3F11F0759165915591459136
:106D7000041B150B260B370B39F318F3E7CFFA92E8
:106D8000EA92DA92CA92BA92AA929A928A927A92E3
:106D90006A925A924A92BA93AA939A938A930895BE
:106DA000FF84EE84DD84CC84BB84AA8499848884A7
:106DB0007F806E805D804C80BB81AA8199818881B3
:106DC000F0E0EC0FFD1FEF0108950E94C3362297FB
:106DD00041E050E060E070E00E94513660F440E035
:106DE0000E94473621F402E26BD03FEF5FC001E220
:106DF00067D03FE75BC0AE010E945E33C801D90196
:106E000043EF54E065E37FE30E94513668F437FBBB
:106E1000AA0FBB1FB395B695A795B7F9088119813D
:106E2000015010400883198340E050E060E87FEB98
:106E300043D02801390140E050E060E87FE33CD0D6
:106E4000A801B901820193010E94C835C801D90186
:106E5000A801B9012FD0280139010881102F110F85
:106E6000110B212F312F0E948F3448E152E761E34B
:106E70007FE320D04801590142E252E964ED7EE30C
:106E80008201930117D04DED5BE96AE27FE316D0F2
:106E9000A201B3010FD044E050E060E070E40ED0F6
:106EA000AC01BD0107D0A401B50108D02296ECE0E9
:106EB0000C94D4360C944F358C019D010C94EE3417
:106EC000E3E3FAE2008351830FEF1FEF2FE708950A
:106ED00001E008950E94BF36EF97EF976A972A87DF
:106EE0003B874887598768017B0100E00B830C834F
:106EF00002C011D21BD20AD2053251F00023C9F7C9
:106F00000B811C81EF96EF966A96E0E10C94D036E7
:106F10000081053221F402D2FED105E2EBCF00E080
:106F20000F830E830A8309833E0102E1600E00E0B5
:106F3000701E09EC14E2088B198B06C0098100232E
:106F400011F400810983EAD1D9D10052B9F3035079
:106F500059F00850B1F3025019F0035049F00CC039
:106F60000A8103950A83EFCF0E8103950E83EBCF41
:106F70000F8103950F83E7CF00810A3279F4AAD1FC
:106F8000AD90BD9098D1BB203AF4B194A19400E0AB
:106F9000B00A0A8103950A83C1D114C0AA24BB2474
:106FA0004AE050E00DC021916F0185010E949A33A3
:106FB000A22EBB24A00EB11E00EDA00E0FEFB01E3E
:106FC000A0D188F30A81002311F000E00F8396D14D
:106FD0000E32F1F4A3D192D10A3231F47BD18D90EB
:106FE0009D9069D19BD117C0882499244AE050E034
:106FF00088D188F421916F0184010E949A33822EF6
:107000009924800E911E00ED800E0FEF901EF0CFA0
:1070100088248A94982C80E071D10C5421F00C5172
:1070200031F0045039F481E0C80E7AD103C001E098
:10703000C00ED81E6BD1E2EDF3E00C947A3680FBE3
:107040005EF44B815C81652F660F660B47D14083F0
:107050005183628363834FCF2B813C813FD1208357
:10706000318349CF37D10D91119625D10A8B2E014D
:1070700003E115D1E0C02ED16D907D901CD1062D7D
:10708000072921F40AED602E04E2702E992022F4E3
:1070900000E1802E07E2902E80E090E001C0019692
:1070A000F30101913F01002319F088159905BCF304
:1070B0000CD12301919581959040680E791EBBC03B
:1070C0000E81002331F0082D092919F49924882410
:1070D000839409EE14E2088B198B0881003739F488
:1070E000F9D0ECD000E1D5D000E0098330C0F1D078
:1070F00046F40D911D912D913D91DDD0C801D9012E
:1071000001C0DCD008810F3611F408E0ECCF053760
:1071100049F70AE0E8CFDDD04D915D9126F46D91FD
:107120007D91C9D005C0C7D0652F660F660B762F3D
:10713000CA01DB0177234AF40DE209839095A095FB
:10714000B09581959F4FAF4FBF4F0AE0A2D03E014F
:1071500007E9600E00E0701E2E0107E9A0D0082F9D
:10716000092B0A2B0B2B11F001E001C000E00D836D
:10717000082D092919F40D8100FF1FC094D0E8895A
:10718000F989E00DF11D0081F30102933F018BD0DD
:10719000C801D901012B022B032B81F799206AF436
:1071A0000F81002351F0A3D010E04501801A910A0D
:1071B00004C000E3F30102933F018E0109561F4F03
:1071C0000619170908151905A4F30E81002399F172
:1071D0000D8100FF30C00881083711F0083549F4EF
:1071E00074D0F3010881008370D000E3F3010083C1
:1071F00022C00F3601F5F30100810033E1F000E316
:1072000002933F0118C00AEF602E04E2702E462C54
:10721000502EF2010081002371F001E040D0F9CF3F
:107220000FEFC00ED01E0DE1602E05E2702E00E2C1
:10723000402E05E2502E420186189708A814B90482
:107240001CF480E090E007C052D0A818B90810E004
:10725000A01AB10AC5010A81002321F401C063D03C
:107260000197EAF70981002339F055D004C053D0C3
:10727000F30101913F015AD00FEF800E901EBAF733
:107280000A81002309F437CE01970AF434CE4BD09B
:10729000FBCF10E00C871D871E871F870895400EC7
:1072A00000E0501E08954C855D856E857F858C01BC
:1072B0009D010C940A34A083B18308958D919D9112
:1072C000A083B183A0E0B0E008950FEF600E701EC0
:1072D000089580FBF701A081B1810895F701A08195
:1072E000B1810D911D91A083B183F80108950981A9
:1072F000002311F001E0089500E00895F6010081F7
:107300000895F601008100530A300895F6010191B5
:107310006F010883089528853985089501E0C00E1E
:1073200000E0D01E08952885398500E2EA85FB85B6
:1073300009950B811C810F5F1F4F0B831C830895E0
:107340000E94CB36C801D9011A013F7740E856E9BF
:1073500068E17BE40E94693638F416D0B38300E01C
:1073600010E020E030E00DC03B2F0E949C340E94D2
:107370008F340AD03383A801B9018C019D010E948A
:107380003235E4E00C94DC36F10100831183228372
:1073900008950E94BF36C801D901BF7741E050E08F
:1073A00060E87FE33B2F0E94513670F440E00E947A
:1073B000473629F40BED1FE029E43FE350C0CC240D
:1073C000DD24EE24FF241CC00BEDC02E0FE0D02ED8
:1073D00009E4E02EF72E40E07FEB082F48D028018B
:1073E000390140E050E060E87FE38C019D013FD02F
:1073F000A801B901820193010E94C835C801D901D1
:10740000AC01BD018C019D012DD02801390144E260
:107410005FEF6BE27CEB26D048E854E466EA7EE35B
:1074200028D048E150EC6FE370E423D045EB1CD04A
:10743000480159014AEE54EB66E870E48201930179
:1074400018D046EB11D0A801B901840195010E9422
:10745000C835AC01BD0106D0A601B70108D0E0E1F6
:107460000C94D0360C944F355DEF68E670E40C94C4
:10747000EE34FDDFA201B301F5CF20E006D0E9F73D
:107480000895259102D0E9F708952D9301501040F9
:10749000202F212B089580E597E7FC010591149199
:1074A000FC013296A591B491FC013496259134915A
:1074B000422F432B19F0F901E4DF01C0DEDF06960D
:1074C00017E78C35910748F3089540E00C94683A2B
:1074D0000E94C7362897802FB32F442E40E050E0FB
:1074E00060E070E00E94513610F401E001C000E05D
:1074F000000F400EBF7743E859EF62E27FE3082FA9
:107500003B2F80D076D041E05CEF6FE777E40E94BC
:10751000693688F5AE010E94A0396BD0042D10E0C9
:107520006BD0488159816A817B8172D0088319832D
:107530002A833B83AE014C5F5F4F2A0140E050E05D
:1075400060E87EE35FD0A2010E94A03940E050E0F5
:1075500060E870E40C811D812E813F8153D0A80129
:10756000B901088119812A813B810E9432350E942C
:107570009C34402E0CC00E949C34602E3DD0A8014B
:10758000B9018C019D0133D0460C03E0402240FA42
:107590003EF4AC01BD0100E010E020E83FE327D05D
:1075A00002E0401608F0B0588C019D0129D0280156
:1075B00039014BEF57ED6EE179E324D045E656E211
:1075C00069E97BEB21D048E554E363EA7DE31CD015
:1075D00041EE5DE565E27FEB17D04BED5FE069ECD6
:1075E0007FE316D00DD02896E8E00C94D8360E94A0
:1075F0003235C801D901089520E030E00C949A3466
:10760000AC01BD010C944F3503D0A201B301FACFF8
:107610000C94EE341B2F6A2FF901A081B181AD01CA
:107620004F5F5F4F408351830C93A62FB12F089576
:10763000BA93AA9324970A831B8389019E012A5F28
:107640003F4F28833983BE01AE014E5F5F4F2AE072
:107650003BE30E946A3720E0AA81BB812C932496E9
:10766000A991B99108950E94C33622974801590102
:1076700041E050E060E070E00E94513698F440E054
:107680000E94473629F400E010E020E030E04EC0D0
:1076900001E2E3E3FAE2008351830FEF1FEF2FE7EC
:1076A0003FE744C0AE010E945E33C801D90145ECFA
:1076B00053E062E47FE30E94EE344AE151E562E187
:1076C0007FE33BD0A801B9018C019D013BD0402E46
:1076D000088100FF14C00A952DD0802F43EF54E09D
:1076E00065EB7FE3042D0E944F3537FB220F331FDC
:1076F000380F3695279537F9C801D9010BC01AD034
:10770000842D912FD90137FBAA0FBB1FB00FB6955F
:10771000A795B7F940E050E060E87EE38C019D0159
:107720000CD0AC01BD01840195010CD02296ECE097
:107730000C94D43642E00C948A330E944F352801D1
:10774000390108950E94C835A201B3010C94EE34AA
:10775000FD0324215C771405212500004E6F726D16
:107760006100547572626F005472657368002D2059
:10777000504C454153452057414954202D20004647
:10778000256420202020203C3E2020202020202076
:10779000002020462564203D20256420487A2020B2
:1077A00020202000202020202020202020202020F9
:1077B00020202020002045524153494E4720454576
:1077C00050524F4D212000726164696F646F6D2EBD
:1077D00075636F7A2E727500204B504F54332D34E1
:1077E000382D547572626F27002A2A2A2A204B5599
:1077F0003D2564202A2A2A2A2A002A2A2A2A2A2AD5
:107800002A2A2A2A2A2A2A2A2A2A0054582025647F
:10781000487A202025646D4120200052582025649C
:107820006D5620202020002A25732A2020002020A9
:10783000205475726E20636F696C212020200043F4
:107840006F696C20626C3F2059657320272B2700DD
:107850002020202020202020200020256425644690
:10786000256425630025642C256420002B253032F7
:10787000645B00253032645B0023005D5325642582
:107880006446256425630025642C25645620002564
:10789000646D562000202020202020203C3E202007
:1078A0002020202020005572783D25646D56202030
:1078B0002E2E2E2E2E2E20002A5A65726F5F4164C6
:1078C00063203C25643E20202000556261743D25E4
:1078D000642E256456202E2E2E2E2E2E2000506F24
:1078E0007765725F42617420203C25643E2000462B
:1078F00025645B25646D415D2020256420202020C7
:10790000002A467265715F5458202564487A200029
:107910004625645B25646D565D20200020413D2591
:1079200064202020002A436F696C20626C2E202581
:10793000633D256425632020002A466572726974C0
:1079400065202020200025633D256425632020003C
:1079500047726F756E6420626C2E20002B256420A8
:10796000202020002D2E2E2E2E2E2E2E2E2B005699
:107970006F6C756D652020202020202020202000A5
:107980002564746F6E652000426565707320202049
:1079900020202020202020200025642020202020BE
:1079A0002D2E2E2E2E2E2E2E2E2B00496E64696328
:1079B0002E20202020202020202020200025732081
:1079C0002D2E2E2E2E2E2E2E2E2B004D6F6465204A
:1079D000202020202020202020202020002B256473
:1079E000202020202D2E2E2E2E2E2E2E2E2B00430C
:1079F0006F6E74722E202020202020202020202036
:107A00000025646D41202000506F7765722E202084
:107A100020202020202020200025646D56202000DA
:107A20004761696E20202020202020202020202057
:107A300000256420202020004850462020202020BF
:107A400020202020202020200038363432302F30D3
:107A5000313233343536373839002020202825306C
:107A60003264293C253032643E202020202000470B
:107A7000726F756E6420626C2E2D4572726F72008B
:107A800047726F756E6420626C2E202D4F4B2D2037
:107A9000002020202A2A2A202564202A2A2A202081
:107AA0002020002B30305B200020204E6F204665C8
:107AB000727269746521202020002054616B65205A
:107AC00046657272697465212020002020202020E4
:107AD0004572726F7221202020202000202020205B
:107AE00020204F4B2120202020202020002020205B
:107AF0002020206C6F6E6720202020202020002C6A
:107B00000130313233343536373839414243444518
:107B10004600286E756C6C20706F696E74657229F2
:107B20000030313233343536373839616263646559
:107B30006600464C4F4154533F2077726F6E67206A
:107B4000666F726D617474657220696E7374616CB6
:097B50006C656421003F3F3F0019
:0400000300000000F9
:00000001FF
